:1000000055AA55AA0200000036700000000000004A
:1000100037F20000000000000F6000000000000048
:1000200000000000000000000F600000007B0000E6
:10003000000800000000000000000000950DE6E64A
:10004000B73214E4BF1E000048CDEB1B40E1FFFFB8
:1000500000021000E100000033660000FD01000016
:100060004902000095020000E102000000000000CB
:100070000000000000000000000000003B660000DF
:1000800043660000000000002D0300004B660000E6
:10009000536600005F66000067660000736600003C
:1000A0007F6600008B660000936600009F6600007C
:1000B000EB6600003B030000AB660000B366000087
:1000C00000000000C3660000ED660000EF6600005F
:1000D000FB660000FD660000FF660000DB660000B6
:1000E000E3660000CB660000D366000001670000F5
:1000F000036700000F670000BB66000000000000FF
:1001000000000000000000000000000000000000EF
:1001100037F2000001000140000000000000000074
:1001200000000000000000000000000000000000CF
:1001300000F002F800F068F80AA090E8000C824491
:100140008344AAF10107DA4501D100F05DF8AFF26E
:10015000090EBAE80F0013F0010F18BFFB1A43F0A5
:10016000010318479C760000CC7600000A444FF04B
:10017000000C10F8013B13F0070408BF10F8014B06
:100180001D1108BF10F8015B641E05D010F8016B4B
:10019000641E01F8016BF9D113F0080F1EBF10F8AF
:1001A000014BAD1C0C1B09D16D1E58BF01F801CBD2
:1001B000FAD505E014F8016B01F8016B6D1EF9D555
:1001C0009142D6D370470000103A24BF78C878C156
:1001D000FAD8520724BF30C830C144BF04680C604D
:1001E000704700000023002400250026103A28BF95
:1001F00078C1FBD8520728BF30C148BF0B60704799
:100200001FB51FBD10B510BDDFF80CD0FFF7F8FF0C
:1002100006F039FB06F052FF0002100003B4FFF7AE
:10022000F1FF03BC06F054FF40BA7047C0BA7047F4
:1002300072B6784600F10A004DF8080C62B630BF7D
:1002400000BF704740BA7047C0BA704711484FF0BE
:100250000F0100F8011B4FF0010100F8011B4FF0E6
:10026000020100F8011B4FF0000100F8011B00F82B
:10027000011B00F8011B00F8011B00F8011B1EF018
:10028000040F0CBFEFF30880EFF309804FF0020179
:1002900005F0D6B80002002011484FF00F0100F819
:1002A000011B4FF0010100F8011B4FF0030100F8A2
:1002B000011B4FF0000100F8011B00F8011B00F8C2
:1002C000011B00F8011B00F8011B1EF0040F0CBFFE
:1002D000EFF30880EFF309804FF0030105F0B0B8A9
:1002E0000002002011484FF00F0100F8011B4FF0F1
:1002F000010100F8011B4FF0040100F8011B4FF051
:10030000000100F8011B00F8011B00F8011B00F8B8
:10031000011B00F8011B1EF0040F0CBFEFF3088057
:10032000EFF309804FF0040105F08AB800020020C5
:1003300011484FF00F0100F8011B4FF0010100F8C8
:10034000011B4FF0050100F8011B4FF0000100F800
:10035000011B00F8011B00F8011B00F8011B00F84D
:10036000011B1EF0040F0CBFEFF30880EFF30980B0
:100370004FF0050105F064B80002002000B506F05A
:1003800077F95DF804EB00F02FB81EF0040F0CBFF6
:10039000EFF30880EFF309804FF0000105F050B84B
:1003A0000A484FF0FF0101704FF0000080F3118800
:1003B0004FF0000080F3098805484FF002010170FA
:1003C00062B604484FF080510160704722ED00E0B2
:1003D0007D05100004ED00E002484FF080510160FF
:1003E0007047000004ED00E04FF0200080F311881A
:1003F000EFF3098098B112480068124909688842F1
:1004000017D0EFF309800E49096820E9F00F8860E2
:1004100000B50B48006806F00AFB5DF804EB0848DD
:1004200008490A68026000688168B1E8F00F81F34A
:1004300009884EF0040E4FF0000080F311887047D9
:100440008005100084051000EFF311804FF02001AB
:1004500081F31188704700004FF0000080F311888D
:100460007047000062B6704772B6704710B5022040
:1004700000F00AFA032000F007FA042000F004FA62
:10048000052000F001FA062000F0FEF9072000F038
:10049000FBF9082000F0F8F9092000F0F5F90F2029
:1004A00000F0F2F94FF00051002001F84A0F887176
:1004B000F022CA710F224A70F94908628862086303
:1004C000886008618861C8604861C8614862C86224
:1004D00048630621022000F0F6F90621032000F00F
:1004E000F2F90621042000F0EEF90621052000F0C3
:1004F000EAF90621084600F0E6F90621072000F097
:10050000E2F90621082000F0DEF90421092000F0BC
:10051000DAF906210F2000F0D6F9022000F0C8F920
:10052000032000F0C5F9042000F0C2F9052000F016
:10053000BFF9062000F0BCF9072000F0B9F9082047
:1005400000F0B6F9092000F0B3F9022000F091F9AB
:10055000032000F08EF9042000F08BF9052000F054
:1005600088F9062000F085F9072000F082F90820BC
:1005700000F07FF9BDE81040092000F07AB94FF093
:100580000051C98C4FEA90100A06C54901D5C54AE9
:1005900000E0C54AB2FBF0F0086070474FF0005031
:1005A00090F84A00000700D0012070477047BF490B
:1005B00000200860BA498860C8607047B84AD160B6
:1005C000642148430A2190FBF1F0B0F5803F06DB3F
:1005D000A0F57F40FF3890604FF6FF7002E00021E9
:1005E00080B2916000F07FB9AD4910B58868B0F570
:1005F000803F06DBA0F57F40FF3888604FF6FF7034
:1006000003E030B10022C0B28A60BDE8104000F0C3
:100610006AB9CA68FFF7CBFF12B1BDE810401047B6
:100620000020FFF7C3FF10BDA0490020091D08608E
:100630009B49086148617047994A51616421484368
:100640000A2190FBF1F0B0F5803F06DBA0F57F407A
:10065000FF3810614FF6FF7002E0002180B2116197
:1006600000F04BB98E4910B50869B0F5803F06DB44
:10067000A0F57F40FF3808614FF6FF7004E00028C6
:1006800006DD002280B20A61BDE8104000F035B9F5
:100690004A69FFF7C9FF12B1BDE8104010470120B9
:1006A000FFF784FF10BD81490020083108607C49B4
:1006B0008861C86170477A4910B58869B0F5803F94
:1006C00006DBA0F57F40FF3888614FF6FF7003E03E
:1006D00030B1002280B28A61BDE8104000F017B945
:1006E000CA69FFF7E0FF12B1BDE8104010470220D1
:1006F000FFF75CFF10BD6D490020103108606849AC
:10070000086248627047664910B5086AB0F5803FD4
:1007100006D3A0F57F40FF3808624FF6FF7003E074
:1007200030B1002280B20A62BDE8104000F0F9B892
:100730004A6AFFF7E0FF12B1BDE8104010470420FD
:10074000FFF734FF10BD59490020143108605449A7
:100750008862C8627047524AD162116848430A21D0
:10076000B0FBF1F0B0F5803F06DBA0F57F40FF382D
:1007700090624FF6FF7002E0002180B2916200F0BB
:10078000DBB84FF00050B0F85A00454909690844F9
:100790007047434910B5886AB0F5803F06D3A0F58D
:1007A0007F40FF3888624FF6FF7003E030B10022CF
:1007B00080B28A62BDE8104000F0BEB8CA6AFFF796
:1007C000C2FF12B1BDE8104010470520FFF7EEFE52
:1007D00010BD4020C10581F8210070473348002139
:1007E0001C3001604FF000524FF6FF71A2F8661006
:1007F0000121016070472D4900201C3108607047BD
:100800004FF0005090F82110C90606D510F8211FAE
:1008100021F010010170012070470020704710B5D1
:1008200004460F2000F044F80F2000F022F81C4886
:1008300044604FF00050C18C090602D54EF660218D
:1008400001E04AF6C871416518490120B8310860D5
:10085000091D086010BD10B50F2000F015F84FF00D
:100860000050C06C0E4920F07F404968BDE8104040
:10087000084700F01F02012191404009800000F16B
:10088000E020C0F80011704700F01F0201219140E4
:100890004009800000F1E020C0F88011704700009E
:1008A00000021000C0270900D0DD06004009002228
:1008B00000F01F02012191404009800000F1E0207A
:1008C000C0F88012EAE74907090E002806DA00F0AE
:1008D0000F0000F1E02080F8141DDFE700F1E020B8
:1008E00080F80014DAE71A4900220A604FF000523B
:1008F000A2F8580001200860D0E715490022091D20
:100900000A60CA06A2F85A0001200860C6E710492A
:10091000002208310A608A06A2F85C000120086003
:10092000BCE70B49002210310A604FF00052A2F8D8
:10093000600001200860B1E70549002214310A6017
:100940004FF00052A2F8620001200860A6E7000004
:100950004009002210B55B4C002020605A4800F08E
:100960009BFD0120206010BD10B54FF0E0214FF03D
:100970008060C1F88001C1F880025449A02081F84C
:100980000004FFF7E7FF4FF00051C88CCA8C00F05D
:100990000300120600EB400001D54D4A01E04C4A2D
:1009A000303A12F8203001F8983F02EB800042788C
:1009B0004A7082788A70C278CA7002790A71427964
:1009C0004A7182798A71C279CA71027A0A72427A4C
:1009D0004A72827A8A72C07AC87210BD70B54FF0BE
:1009E000005400F07F00049D84F88D0084F88E1080
:1009F000A4F8942001213748002283B1C0F8801167
:100A000094F8913023F0700384F8913094F8913089
:100A1000702606EA05152B4384F8913001E0C0F8F2
:100A2000802114F8923F23F034032370C0F844224D
:100A3000C0F84012D0F89C110129FBD170BDF0B56F
:100A40004FF00054DDE90765DDE905C700F07F00E0
:100A500084F88D0084F88E10A4F8942084F88F30E8
:100A6000A4F896C001211B48002287B1C0F880116C
:100A700094F8913023F0700384F8913094F8913019
:100A8000702707EA05152B4384F8913001E0C0F880
:100A9000802114F8923F23F034032370237843F02D
:100AA0002003237016B1C0F8481201E0C0F84822B4
:100AB000C0F84422C0F84012D0F89C110129FBD1A3
:100AC000F0BD000084140022AA8206001AE000E0B3
:100AD000147100000010002237480121016000213C
:100AE00001607047354801210160002101607047B5
:100AF00000B54FF0E0230122C3F8802103F5C07355
:100B0000FFF7F0FFFFF7E8FF2C4808380260A0204D
:100B100083F88002C3F8002143F8802C00BD2749E8
:100B2000083910B10020086070470120FBE7234816
:100B300001217838016000210160704710B572B65C
:100B40001F490C78002104E01D4A521C525C42549B
:100B5000491CA142F8DB40F6FC0000F09DFC62B6A7
:100B6000204610BD144901201C3908607047144804
:100B700020300078124921310978401A00F03F00F6
:100B800070474FF00051027881F80022427881F8D6
:100B90000122827881F80222C27881F80322027948
:100BA00081F80422427981F80522827981F80622AF
:100BB000C07981F8070270475C8400229405002206
:100BC0000004002010B50A2000F05AF80B2000F0B5
:100BD00057F80A2000F05FF80B2000F05CF80521C0
:100BE0000A2000F063F805210B2000F05FF84FF0B9
:100BF00000507F2100F8351F4170C1700021C17184
:100C000001724172817210BD01238340D8B24FF04E
:100C10000053002993F8361001D0014300E08143CE
:100C200083F8361013F8381F0AB1014300E08143FE
:100C30001970704701238340D8B24FF00053002948
:100C400093F83C1006D0014383F83C1093F83E1013
:100C5000014305E0814383F83C1093F83E10814343
:100C600083F83E1013F83D1F22B1014319709978A3
:100C7000014303E08143197099788143997070476B
:100C800000F01F02012191404009800000F1E020A6
:100C9000C0F88011704700F01F0201219140400907
:100CA000800000F1E020C0F8801270474907090E6B
:100CB000002806DA00F00F0000F1E02080F8141D93
:100CC000704700F1E02080F8001470477047FE4B39
:100CD000FE4A998A814203D2401AD080084601E038
:100CE0000021D180DA68FA491047F74810B5006949
:100CF0008047F649C88810B1BDE81040E7E7896829
:100D0000002903D0BDE810400120084710BDEE487F
:100D100010B500698047ED4C4FF00000A16819B193
:100D200088470020A06010BDFFF7D0FF10BDE74945
:100D3000CA780B7952005A43E34B0878D2B29B68C9
:100D400040F48070C968184701461822DE4806F052
:100D5000BBB838B5DD4A8179132311714179D1705F
:100D6000027901F0070102F01F028DF800208DF8D2
:100D70000110C078032200F01F008DF80200D24855
:100D8000694644681846A04738BDF8B50446007C5B
:100D9000CD4DC0F34002014662F35F01C0F3800213
:100DA00041EA8201C0F3C00241EAC201C0F300126D
:100DB00041EA0211C0F3401241EA42118DF80010DD
:100DC0008109607C272300F0010241EA0211C0F38F
:100DD000400041EA40108DF80100607CC0F38001C2
:100DE000C0F3C00241EA0211C0F3001241EA42110D
:100DF000C0F3401241EA8211800941EAC0108DF827
:100E000002006E68032269461846B047E0792B233A
:100E1000C0F38002014662F39F01C0F3C10241EAC0
:100E20000211C0F3401041EA80108DF80000607C90
:100E3000A17CC00901F0030140EA01108DF8010016
:100E40006E68022269461846B0472D262B6801229B
:100E5000694630469847A17C9DF80000C1F38001A7
:100E600008438DF800006B680122694630469847B8
:100E7000F8BD10B50446FFF76CFF204600F04FF9AF
:100E80002046BDE8104080E738B53D218DF80010C0
:100E90008D49044612204B68012269469847A08874
:100EA000FFF715FF38BD10B5044600F07AF920466B
:100EB000BDE81040E8E7F8B5834C122506462368E4
:100EC00001226946284698479DF80000012240F01B
:100ED00008008DF800006368694628469847482551
:100EE000236801226946284698479DF800000122A0
:100EF00020F0060040EA46008DF80000636869466D
:100F000028469847236801226946284698479DF855
:100F10000000012240F001008DF80000636869467E
:100F200028469847F8BD38B5674D482401222B68FC
:100F30006946204698479DF80000012220F00100F4
:100F40008DF800006B6869462046984738BD38B573
:100F50005D4D2A2401222B686946204698479DF85A
:100F60000000012220F0100040F001008DF8000088
:100F70006B6869462046984738BD38B5524D2A24DB
:100F800001222B686946204698479DF800000122FF
:100F900020F001008DF800006B68694620469847F4
:100FA00038BDF8B5484C44250646236801226946F9
:100FB000284698479DF80000012240F082008DF8F5
:100FC000000063686946284698472D25236801225A
:100FD0006946284698479DF80000012220F0FC0051
:100FE00040F08E008DF800006368694628469847F7
:100FF0001425236801226946284698479DF8000079
:10100000012220F0070040F001008DF80000636825
:1010100069462846984715252368012269462846CF
:1010200098479DF8000006F01F0120F01F000143C3
:101030008DF8001063680122694628469847F8BD7C
:101040002DE9F843204C132517468846814623682E
:10105000012269462846984701269DF8000006FAB5
:1010600008F120F01F0001F01F0101438DF800106E
:101070006368324669462846984727252368012237
:101080006946284698479DF80000BE4020F03F0082
:1010900006F03F0101438DF80010636801226946A4
:1010A000284698472E2523680122694628469847F6
:1010B0009DF80000012240F00C008DF800006368EC
:1010C00069462846984705E0900510003802100050
:1010D0009B0C00003E2023680122694698479DF83A
:1010E000000000F0300189F80010BDE8F883554B8E
:1010F00040F480701B681847524B40F480705B6866
:10110000184701B506209DF80010012201F01F01CB
:101110008DF800104B494B686946984708BDFEB5ED
:10112000494D04460078287060786870454EA07874
:10113000A870312733680122694638469847E0791C
:1011400040069DF8000002D540F0200001E020F0AC
:1011500020008DF80000E179090602D540F08000FA
:1011600001E020F080008DF80000736801226946DC
:101170003846984721893220C1F30801ADF80010A4
:10118000E168CDF8021029788DF8061069788DF89D
:101190000710A9788DF808107368092269469847E6
:1011A000FEBD70B504460168274886B0254D8160B4
:1011B000A168C160E1680161217C162001F0010194
:1011C0008DF80010617C8DF80110A17C8DF8021063
:1011D00000218DF80310A18A0F22C1F30C01ADF894
:1011E0000410E18AC1F30B01ADF80610218BC1F3A5
:1011F0000B01ADF80810618BC1F30B01ADF80A10BB
:10120000A18BC1F30B01ADF80C10A17F8DF80E106E
:101210006B686946984731262B68012204A930463D
:1012200098479DF81000E17F20F01F0001F01F019A
:1012300001438DF810106B68012204A930469847CD
:1012400006B070BD90051000380210004FF0E0218C
:101250004FF48030C1F88001C1F880027249A020AB
:1012600081F80004704730B5704C01252560E50613
:1012700003F03F0385F86B30002304E051F823505E
:1012800040F823505B1C9342F8DB0020206030BD07
:1012900030B595B00446302105F072FE6448006810
:1012A00000906348001D00680190614808300068A4
:1012B00002905F480C30006803905D481030006871
:1012C00004905B4814300068059059481830006855
:1012D000069057481C300068079055482030006839
:1012E000089053482430006809905148283000681D
:1012F0000A904F482C3000680B904D483030006801
:101300000C904B48343000680D90494838300068E4
:101310000E9047483C3000680F90454840300068C8
:1013200010904348443000681190414848300068AC
:1013300012903F483F494C306FF00205006813900F
:10134000009888424DD1A810A06120612060A06261
:10135000E062E061206203A8029900F06FF8019951
:1013600081423ED10B9845F2AA5180B2884208D101
:101370000498C0B2A061139A92B28A4200D0801D34
:10138000E0610C9880B2884217D10398039A00F468
:101390007F40D2B240EA0240039AC2F307421043B0
:1013A000254A904203D30598C0F3012000E00020B5
:1013B0002061059800F00F0020600D9880B28842EF
:1013C00001D10698A0620E9880B2884201D1079898
:1013D000E0620F9880B2884201D10898206215B06F
:1013E00030BDA56125612560A562E562E5612562E4
:1013F000F5E710B50446142105F0C2FD0C487C3811
:10140000006820600A4880380068606008487838C2
:101410000068A060064874380068E06004487038CE
:101420000068206110BD000010E000E0441B0022B5
:10143000B41E04005C000D6000010200F0B5074618
:1014400000200346184E10E057F8235003224FEABD
:10145000C20C45FA0CF484EA2064E4B2521E56F839
:10146000244084EA0020F2D55B1C8B42ECDBF0BD0B
:1014700070B5054600200C4C0246103C09E0AB5C00
:10148000521C03F00F0604EB1313A65D1B783044C7
:1014900018448A42F3DB70BD08B50090401E0090EE
:1014A0000028FBDC08BD0000547100004FF0005123
:1014B000C88C4C4A00F0030012687AB101280AD0A7
:1014C000022806D0032802D04FF416700EE0462002
:1014D0000CE096200AE04FF4967007E001280ED049
:1014E00002280AD0032806D04FF4E170401E21F8EC
:1014F000520F088070473220F8E76E20F6E7DC20B4
:10150000F4E748F61971480720F82A1F0B2180F8E4
:101510003E1000214183022180F8C0104FF0085195
:101520000120C1F8D4032F49983908602E4908607A
:1015300070474FF0005141F29840C884B6E74FF031
:10154000005140F29A70C884B0E74FF00050C08C50
:10155000A0F5A051983901D00020704701207047B4
:101560004FF000518A8C60F304028A8470471F4850
:10157000016841F00401016070471C48016821F0D6
:101580000401016070474FF000510881704717490E
:10159000283109680160154918310968416013490B
:1015A0001C3109688160114920310968C1600F4907
:1015B0002C31096801610D490C39096841610B49F9
:1015C00014310968816170474FF00050808870477E
:1015D0004FF00050807970474FF000514C2081F857
:1015E00020007047DC040022EC1B002210ED00E01C
:1015F00030B41DC8484981E81D00012130BC0020DD
:1016000005F046BA2DE9F84F44480124006810F867
:101610006C5F417890F846004D4300F0030004FAF7
:1016200000FA3D486421103005F0AAFC3C4804F063
:10163000D9FD3B483B490471097809B90221017180
:10164000DFF8D480002408F1100B36E0DFF8D090EA
:10165000032735490026C9F80010484604F0C6FDA6
:1016600000226B460121104605F062FA012100209C
:1016700005F03DFA98F8000060B103F014FF7F1EFA
:10168000002F0AD0E9DC76B34FF000005946D8F8B5
:1016900004200FE04FF00106F5E74FF0040004F0DE
:1016A0009AFDF0E751F8203032F910703B4441F8D0
:1016B0002030401CA842F5DB641C5445C6DB012EDB
:1016C00011D1164900205C46184A0B6809E093F8CE
:1016D000B26054F8201006F00306314122F81010D1
:1016E000401CA842F3DB124901200870BDE8F88FC6
:1016F00010B50446002005F07CFA022005F079FAC6
:10170000E00701D0FFF77EFF022005F08DFABDE86B
:101710001040002005F088BAA805100054051000FC
:101720004C02100079051000A1150000B0580120EE
:101730008C02100010B51C4C40F2FF112068FFF71E
:101740007DFE2168C1F8FC07FFF748F800213F2023
:101750000EF17EFAFFF742F82168BDE810403F2302
:101760004FF400721148FFF77EBD10B540F2FF3113
:101770000F48FFF763FE0E49C1F8FC0FFFF72EF884
:1017800000213D200EF164FA00213E200EF160FAA6
:10179000FFF724F8BDE810403D234FF48062044970
:1017A0000448FFF760BD000054051000F0EF03008F
:1017B00050000120F0CF030030B41DC84F4981E82C
:1017C0001D00012130BC002005F062B910B50020D9
:1017D00005F00FFAFFF7BBFB00F064F80446FFF7D3
:1017E000CCFB012C04D13C224549A020FFF77FFC13
:1017F000002005F019FA012010BD10B5FEF714FF06
:10180000BDE81040822003F061BE2DE9F0470020C2
:1018100005F0EFF900253B4F4FF0360A6E1EA84643
:10182000E8B2FFF76EFC0020FFF745FB3C68386824
:10183000A042FCD03868A042FCD133496420FEF7B6
:10184000FBFEFEF79EFF81463868A042FCD0386858
:10185000A042FCD1FEF795FF0446FFF764FBFEF7BC
:10186000E3FEA9EB040080B2B0EB0A0001D401460C
:1018700000E04142B14204D2002800DA404206466C
:10188000A8466D1C6DB2202DCADB1D4908F0FF0073
:10189000743981F8B000FFF734FCBDE8F047002050
:1018A00005F0C2B9FEB50025684604F09BFC174858
:1018B00000900320114E8DF804000446684604F0A1
:1018C00095FC002202AB0121104605F031F90121FF
:1018D000002005F00CF9307838B1641E03F0E3FD08
:1018E000002C05D0EADC2846FEBD4FF00105FAE7E2
:1018F0004FF0020004F06FFCF5E700001C0610003A
:10190000C4000120981B0022AB17000069170000DB
:1019100030B41DC88E4981E81D00012130BC002073
:1019200005F0B6B82DE9F84F8A48006810F86C4FFA
:1019300040784443FEF75FFF85486421103005F08E
:101940001FFB3221844805F0F9FA3221834805F063
:10195000F5FA814842F21071323005F0EFFADFF803
:10196000F8A10020AAF1320A47F6FF71AAF1320B62
:10197000CA4304E02AF810102BF81020401CA042A3
:10198000F8DB774804F02EFC75490120002508712A
:10199000DFF8CC9103267349DFF8B4810027C9F83A
:1019A0000010484604F022FC00226B46012110463C
:1019B00005F0BEF80121002005F099F898F8000024
:1019C000C0B103F070FD761E002E16D0E9DCBFB367
:1019D0006148D8F8041005FB04F200F13200DFF88A
:1019E000708100EB42034FF0000056465F4608F15D
:1019F000100823E04FF00107E9E74FF0040004F07E
:101A0000EAFBE4E731F8102023F8102058F82020F2
:101A100031F910C0624448F8202031F9102037F91C
:101A200010C0624501DD27F8102031F9102036F989
:101A300010C0624501DA26F81020401CA042E1DB0C
:101A40006D1CC82DA4DBDFF808810020C821424DA1
:101A500052465B4608F110080EE033F9106032F987
:101A60001070F61B761025F8106058F8206096FB71
:101A7000F1F648F82060401CA042EEDB364F002013
:101A8000364E3237894615E0002258F8203011468C
:101A900001FB040C37F91CC0BCEB030C01D5CCF1E5
:101AA000000C491C6244C829F2DB92FBF9F126F8CC
:101AB0001010401CA042E7DB002707E036F9172092
:101AC00035F91710F8B203F004FF7F1CA742F5DBCD
:101AD000BDE8F84FFEF782BE2DE9F84300248DF8EB
:101AE0000040FEF788FE002005F083F8194D2868B5
:101AF00090F86B00FFF755FA2F680025A1464FF0CC
:101B00000108A1370024785D08FA04F68DF80090EA
:101B100006400DD0224629466846FFF791FA9DF807
:101B20000000202804D132462946052003F0CEFDCE
:101B3000641CE4B2062CE6D36D1CEDB2052DE1D396
:101B4000002005F071F8FEF749FEBDE8F8830000BB
:101B50002C06100054051000B4100120F6370120A7
:101B600054021000C118000010B5044602210020E4
:101B700004F08EFF0F48046010BD08B50E48FEF754
:101B80004EFE00226B460221104604F0D1FF0221D6
:101B9000002004F0ACFF09485522016805480A718D
:101BA00000684871020A8A71020CCA71FEF7E7FCEC
:101BB00008BD00005C021000191B00005805100051
:101BC00008B50024DFF85881564F4FF400492646E7
:101BD00000226B464146104604F0AAFF009880039D
:101BE00019D5FEF741FC504804680660FEF73AFC40
:101BF000E00701D0FFF709FEA00701D5FFF7E6FDDA
:101C000000231A460121022003F04AFE4FF400315E
:101C1000002004F06CFF0098000411D500256D1C15
:101C2000EDB2FFF7D3FD01286ED0032DF7D90022C6
:101C30004946082003F04AFD4946002004F057FFBA
:101C40000098000510D53948046806602046FFF763
:101C50004FFD4FF40061002004F049FF0023E1B282
:101C60001A46062003F01CFE0098C0040CD5FFF7AE
:101C700084FF002301221946022003F011FE4FF4D5
:101C80008051002004F033FF0098800406D5FFF750
:101C900051FD4FF40051002004F029FF009840044A
:101CA00006D5FFF762FD4FF48041002004F01FFFCE
:101CB0000098400311D5386890F8A000C0070CD0F8
:101CC000FFF70AFF4FF48021002004F010FF0023EB
:101CD0001A4619460C2003F0E3FD009800037FF537
:101CE00077AF386890F8A0008007F8D5FFF71AFEA4
:101CF0004FF40021002004F0FAFE00231A46194692
:101D00000E2003F0CDFD63E70120FFF7F1FCE1B207
:101D10000023C4F30722082003F0C2FD8CE7000073
:101D200003F80F0054051000740510007005100032
:101D300010B58143C80711D06448016841F0010122
:101D400001604FF40061002004F0A2FE0122002394
:101D5000BDE810401146052003F0A2BD10BDFEF7FE
:101D6000F2BC10B5FEF7EFFC0121BDE810400846BB
:101D700004F08EBE5649012805D0022805D003285C
:101D800005D1042002E0022000E003200870704723
:101D900038B5002004F02DFF4E48006810B1FFF761
:101DA000E9FF01E000F0CCF949484B4900780228EE
:101DB00013D003280ED0042812D001240025FEF7EA
:101DC000D6FE00B101256946032004F0A0FE00986C
:101DD00058B909E00868847AF0E70868447AEDE7C2
:101DE0000868B0F80B40E9E715B1142C00D21424B0
:101DF00020463A49FEF7AFFC0324394D00F043FA80
:101E0000012807D1287858B1641E03F04CFB002C40
:101E10000DD0F3DCBDE838404FF0000004F004BF03
:101E2000304801683048006800F01CF9F2E70320F0
:101E300004F0D1F9EEE770B52C4804682C490D6820
:101E40000C6095EA040F27D0214E2DB1A4B1214694
:101E50002846BDE870406BE7022030701E480068DD
:101E60000079000701D40420307021462846FFF78E
:101E70005FFFBDE870408BE7FEF765FC0121084677
:101E800004F035FE0120307021462846FFF750FF50
:101E9000BDE8704000F0F7B870BD10B5FEF753FC18
:101EA0000121084604F023FE09490420087000F0CF
:101EB000B1F8BDE810406BE710B5FEF744FC012116
:101EC000084604F014FEBDE8104061E770051000FC
:101ED000700210006805100054051000131D00006A
:101EE000A00610007C0210007802100060051000AF
:101EF000740210002DE9FC5F0E4600281BD05549E6
:101F00000978042917D1002A15D1DFF84C91DFF8A0
:101F10004C81534DD9F800109246097A49070ED5E5
:101F2000A978491CC9B2A970032906D8018808EB11
:101F3000460020F8021CBDE8FC9F85F802A00320A3
:101F400004F057FE454801906C78B5F904B0287844
:101F5000274640B941480F235A460094801D0199F5
:101F600003F059FF002734B93C4A5B46921D901D8F
:101F7000019903F041FF39496F700C31B5F9042024
:101F8000B5F90630002007E031F910409C4201DD30
:101F9000012404E0401CC0B29042F5DB0024032081
:101FA00004F042FED9F8000090F8E307DA2823D1C4
:101FB000D8F80010C8F81210B8F80410A8F81610D5
:101FC000D8F80610C8F81810B8F80A10A8F81C10AD
:101FD000D8F80C10C8F81E10B8F81010A8F8221085
:101FE0001E48C8F824A0C8F828A01230A8F82CA0D1
:101FF0004682A9788182C4822C70002C9BD0FFF786
:10200000AEFEBDE8FC5F0121084604F041BD144866
:1020100000787047124A012050700F480068017A1A
:102020004B0790F8711002D590F86C3001E090F8F1
:10203000703059439180B0F84B00D08000210748A0
:1020400011709170C1600182C0F80610418100F0EA
:1020500017BBDFE77002100054051000283801207C
:102060006002100070B5054630480C46224690F9D3
:102070000D102F484068FFF73DFF21462846BDE878
:10208000704000F014B810B5032004F0B2FD4821F0
:10209000284804F075FF274901200870032004F048
:1020A000C3FD0121BDE81040022004F0F1BC2DE980
:1020B000F041DFF884800746002698F800000D46BE
:1020C00004282CD047EA0504032004F092FD194AA5
:1020D000174B978115619868506098F800000428A4
:1020E0001FD0FF2111751070E0070DD01348016853
:1020F00011F86C0F49784843906042000D485968C8
:10210000163004F09CFE0126032004F08DFD002E05
:1021100009D0BDE8F0410121022004F0B9BC0C4611
:10212000D2E7197BDEE7BDE8F0810000E40610008D
:10213000A0061000280710007002100054051000BF
:102140002DE9F0418A4C0026DFF82882207802270A
:10215000894D04280ED000F001FD012819D08748D0
:10216000237802680320022B517B10D198F80030AD
:1021700093B113E0FFF74BFF012803D098F800005C
:10218000012804D17E49277001202E600870BDE827
:10219000F08127702E60FAE7917B0420127AD30732
:1021A00001D19207F3D52A68521C2A608A42EEDDDB
:1021B0002E602070EBE730B41DC8724981E81D0025
:1021C000082130BC012004F063BC2DE9F0416B48CC
:1021D00000250068C17BC90753D06B49664E2F4666
:1021E0000978C90748D0DFF888810125002498F8CC
:1021F0000010664A022904D0032914D0042921D1F1
:102200000FE090F8241192F90030994205DB90F923
:102210001C1192F90020914201DD847C12E0447C83
:1022200010E0447D0EE090F8241192F900309942BC
:1022300005DB90F91C1192F90020914201DD047D2B
:1022400000E0C47C00F08AFC012804D050480078EB
:10225000012807D00AE098F80000042806D00025DD
:10226000776006E098F80000022807D07068401CEC
:1022700070607068A04203DD776002E07760F8E785
:102280000025284683E72DE9FE4339483E4D0126C7
:102290000078404FDFF80081032816D004286846F4
:1022A00010D0002403F09EFFFFF78FFF2978C907A5
:1022B00000D0012440EA0401C90716D02D4909784D
:1022C00001B310E000F02EF812E06846002403F09D
:1022D00089FFFFF77AFF2978C90700D0012440EA77
:1022E0000401C90701D08DF804603860C8F80040C7
:1022F0002A480090684603F079FF012806D00020A4
:10230000BDE8FE8302218DF80410EEE702AB002247
:102310000821012004F00CFC0821012004F0E7FB57
:102320000120EDE770B50446002503F05BFFFFF7E1
:102330004CFF1249C3074FF0020205D00968C97B60
:1023400089070FD504210BE00F4B1B78DB0700D06A
:102350000225AB0707D50968097A490702D5052187
:10236000217100E022710B4908600B48056070BDC7
:10237000700210007905100068021000540510006A
:102380008C021000A0061000740210006C051000F2
:102390005C0510007C02100078021000672100002C
:1023A0001C4808B500210122416002708160C160B3
:1023B000491E104604F09BFBFFF74BFE6B460022C4
:1023C0001721012004F0B4FB0098800705D5FFF722
:1023D00032FD0221012004F08AFB0098C00705D0DD
:1023E0000121084604F083FBFFF7D2FC0098400768
:1023F00005D50421012004F07AFBFFF74EFD00987B
:10240000C006DBD51021012004F071FBFFF754FD5D
:10241000D4E70000700210003221914804F08EBD14
:102420002DE9FF4F8F4F064683B0386893468E4A9A
:10243000017C6FF0130C01F00F050121029112785D
:10244000B0F91840B0F91C10C5F110094FF00008A0
:102450004FF0010A012A2DD1C27B92062AD5B0F98C
:102460001E40B0F92010012B02D0022B10D04FE0FB
:10247000C28BCDE90028438C28223C21584603F02A
:10248000A9FB04B23868028CCDE90028838C25E0D2
:10249000028BCDE9002AD046438CE24662460021F9
:1024A000584603F097FB04B23868828BCDE90028C8
:1024B000838C27E0012B02D0022B12D028E0028B64
:1024C000CDE90028C38A28223C21584603F082FB2C
:1024D00004B23868828BCDE90028438B28223C2146
:1024E00012E0018BCDE9001AD046C38AE24662466B
:1024F0000021584603F06EFB04B23868828BCDE9A8
:102500000028438B52460021584603F063FB01B27A
:102510005648554ADFF848A10068137883463F685B
:1025200017E036F910C03AF91020022811D0012B1B
:1025300008D197F80F805FEA886803D5049A32F9CA
:10254000102002E0ACEB020212B2A24215DCCA4239
:1025500013D4401EE5D2029800280ED058465346A8
:1025600009E033F9102036F910106A4301FB092104
:10257000091123F81010401EF3D207B0BDE8F08F08
:102580002DE9F0411C46069F15460E46C00718D09F
:1025900000F0E4FA002814D132480068C07B8007BC
:1025A00003D533480078042806D03B462246294606
:1025B0003046BDE8F04133E73046BDE8F04100F079
:1025C00002B8BDE8F0812DE9F04F2649294C4FF0C3
:1025D000010E0A68DFF888B094F90040117CB2F966
:1025E00018A001F00F0692F86D10C6F11008B2F9AC
:1025F0001C900B4614E093FBF1F7C3EB440501FB81
:102600001737EDB2FFB23BF9155030F9177005EBF3
:102610000A0CBC45B2DBA5EB0905BD42AEDC5B1E76
:10262000012BE8DABEF1000FA8D0DC4614E092F8E6
:102630006D50C1EB440391FBF5F705FB1715EDB2A7
:10264000DBB230F915703CF91350754307FB0855A0
:102650002D112CF81350491E0129E8DA8EE70000ED
:10266000B058012054051000F04F0120140510004F
:102670001005100011051000F54800210160704799
:10268000F34800210160801F8180142141703421B2
:10269000F04804F053BCF04A10B5126801465200ED
:1026A000EE4804F0CCFBEE490120087010BDF0B4F8
:1026B000EC4D944600222E68EB4D144613462D68CF
:1026C000A6B995F91C618E4210DD00210CE030F9AD
:1026D000116095F8BA70BE4201DD641CE4B2FE429E
:1026E00001D55B1CDBB2491C6145F0D395F8BB00FA
:1026F000A04200D213B9984201D204B1012295F848
:10270000BD10F0BCD248801C00F092B92DE9FF4FFB
:102710000746002081B0DFF83893D44C461EDFF81E
:1027200038B3984682460546A9F106090090012A69
:102730000CD1DBF8000039464200C648643804F08A
:102740007EFB89F80180012189F80210C149DBF87C
:1027500000C021F81C8099F80130A3EB0802D3B225
:10276000C14A126892F8BF80984506D8002189F8BE
:102770000210BF49012008704BE099F802000128BF
:1027800047D1DFF8D0B20020ABF1640B0BF1320E71
:10279000894613E037F810802EF810803BF81010AF
:1027A00037F81080A1EB080109B229F81010A142F6
:1027B00001DD0C4646B229440DB2401C6045E9D308
:1027C00092F8BE00984212D9B2F8C000A0420EDAC8
:1027D000117CB6EB111F0AD1B2F8C210A94206DA79
:1027E000029931F91610814201DD4FF0010A92F889
:1027F000E307FE2805D109EB4C0043808680C480A6
:102800000581934892F8C4105246401C00F010F91C
:102810000090009805B0BDE8F08F2DE9F041924B93
:102820004FF0000C65461B686446664693F824E149
:1028300067468E4520DD6046BDE8F08130F9121014
:10284000B3F8B8C0614502DD0D442DB209E011EBCB
:102850000C0F06D593F810C0B2EB1C1F01D00C442E
:1028600024B2B3F818C0CCF1000C614504DA197C2D
:10287000B2EB111F00D00126521EDFD2002C00DA6D
:102880006442AC4201DD06B1012793F8B5103A4627
:10289000BDE8F0416E48C01C00F0CAB82DE9FF4FFA
:1028A00081B090468B4600240220DDF83CA004F065
:1028B000A0F9DFF8B491664F2546D9F80000A7F1DA
:1028C000060690F8B000800711D5694802780570B7
:1028D000CDF800A058460E9B0499FFF717FF044659
:1028E000012801D024B12BE01220307028E07D7047
:1028F000D9F8003093F8B000C00721D04FF0000B9A
:10290000444652465946584608E034F910C093F8F8
:10291000B380C44501DD491CC9B2401C9042F4D3C8
:10292000514501D14FF0010B93F8B4105A46484875
:1029300000F07EF80446012803D11020307013E027
:102940003D708CB9D9F8000090F8B00000070BD5A5
:102950000AF0FF020E990498FFF75FFF0446012872
:1029600003D11420307012E0FD7084B9D9F8000052
:1029700090F8B00040070AD552460E990498FFF728
:1029800096FE0446012803D1132030701DE0BD706F
:10299000DCB9D9F8000090F8B000C00614D535486D
:1029A000007888B134480078012801D0B5800CE067
:1029B000B088401C80B2B080B0F5166F05D91620E3
:1029C000B5803070012400E03D60022004F02CF955
:1029D00020461FE770B506460C7800200870244892
:1029E000214D01210170286890F8B100C00709D07D
:1029F000022004F0FEF83046FFF74DFE022004F0FE
:102A000013F909E01D48016841F0010101604FF42C
:102A10000061002004F03CF828682246012190F86B
:102A2000B100BDE8704000F00103052002F038BF9E
:102A300010B500231C4642B10278521CD2B202707B
:102A40008A4203D90470012300E00470184610BDC7
:102A500086021000B638012014051000B05801207D
:102A60008C02100098021000540510000080FFFF37
:102A70007B05100079051000910210007005100010
:102A800070B5FF4C01200025207065711921FD48AB
:102A900004F054FAFB483221193004F04FFAF94897
:102AA00032214B3004F04AFAF6484FF496710D3853
:102AB00045602561E5606570A5714FF4C87060617F
:102AC000BDE87040F04804F039BAF0B5EF48F04B7B
:102AD00001680020186058601881C3F80A00C3F824
:102AE0000E0001F13F0201F14704588203F10A058B
:102AF0000AE032F8106023F8106032F81060275CAA
:102B0000F61B25F81060401C91F86C608642F0DCE2
:102B1000E048007800280AD0DF480078002806D175
:102B2000D84831F8652F0D38028089784180F0BD92
:102B3000D648006890F8801069B1490010F88C2FD1
:102B4000521C40784A43C2EB022100F01F000141B1
:102B5000CB48018170470121F0E77047C848006900
:102B6000002800D00120704710B5014601248C4098
:102B7000C349C44BC74AC9680020A3F10D030C42E6
:102B80001988127807D1012A04D1C44A1278002A80
:102B900000D0084610BD012AFCD15888081A80B21E
:102BA00010BD02460020012905D0BA4B1B7813B195
:102BB000BA4B1B785BB9B24B01209040DB681842DE
:102BC00001D1B34801E0B2480A3030F812000029C0
:102BD00001D11046C8E770472DE9F0418C46DDF879
:102BE000208004461D461646002741466046FFF7F2
:102BF000D8FF0346A548006890F83A00C00702D005
:102C0000B8F1010F06D034F9160034F915108842D6
:102C10000EDC0AE034F9161034F91520881800B2D9
:102C2000BCF1010F04D1914201DD084600E01046DD
:102C3000984204DD012707FA06F0AF400743384603
:102C4000BDE8F081014600208A0700D0012011F084
:102C50000C0F01D040F0020011F0300F01D040F015
:102C6000040070472DE9FF4315461C460B9F009159
:102C70000397CDE901540E460022814601231146F7
:102C8000FFF7AAFF03970096CDE90154804603237E
:102C9000022201214846FFF79FFF03970096CDE9E6
:102CA000015440EA08080523042202214846FFF7A0
:102CB00093FF40EA080004B0C0B2BDE8F0832DE9FC
:102CC000F0410C46014632226F4804F0B8F86E48D5
:102CD00032227349323004F0B2F86A496A4832222B
:102CE0001931643004F0ABF86649674832224B3141
:102CF000963004F0A4F8634A0020FF230D3A4FF009
:102D0000010E5668674A07465F49156814E00EFAD7
:102D100000F2224201EB400C02D0ACF8C83001E0D6
:102D2000ACF8C870324201EB400202D0A2F8FA308F
:102D300001E0A2F8FA70401CA842E8D380E72DE930
:102D4000F04F00259B469AB0531EDFB22C462B460F
:102D50000DF1340AE94611E031F9136035445E1C87
:102D6000B44695FBF6F629F81360FE1A5B1C31F9A0
:102D70001680444494FBFCFC2AF816C09342EBDB1B
:102D8000BBF1010F01D1921ED2B24C4655460FE065
:102D900034F9123035F91260334403EBD3735B100E
:102DA0001BB2002B04DD31F81260F31A20F8123048
:102DB000521EEDD21AB0BDE8F08F2DE9FE4F304D16
:102DC00082463048894600262C782E703221AF305A
:102DD00004F0B4F814B1BAF8060068812B4F314DF5
:102DE000386890F82A10C9070BD0009490F82B008F
:102DF000514600F00F03288802B22248193003F030
:102E00000AF8022003F0F5FE28881E4900B21931A5
:102E100000904B46224A01F1960002F038FF022052
:102E200003F002FF17493222AF31A1F1320004F062
:102E300006F83868DFF87080C07B000715D51548A4
:102E40000078012811D198F8000070B91348007873
:102E500058B128880B4900B200901448AF3102687D
:102E60000846938E243202F0B6FD286805494200D8
:102E7000AF31A1F1640003F0E2FF0D48007819E0E2
:102E80008C021000F938012000EC012054051000DC
:102E9000B0061000F04F01207805100079051000F1
:102EA000B0580120140510005C05100058051000F2
:102EB0003C051000012806D12888F84A03B2F849D9
:102EC000504602F04EFEF74998F800000978084392
:102ED00031D1386890F82A00400707D5EF492A78A1
:102EE0003231012301F13200FFF729FF386890F8F1
:102EF0002A1089070BD590F86D100091E74990F8DA
:102F00006C3090F82C206431084600F06AFAE349EE
:102F100032226431A1F1320003F091FF2968CDF82B
:102F20000090CDE90114DD4BDD4903F1320250463A
:102F3000FFF7B4FC06463046BDE8FE8F2DE9F041B0
:102F40000025DA4B06462C46681E2A46AE46DFF8B8
:102F500058C31F680CE036F912308B4202DA0B447A
:102F6000002B04DC012536F9124050B203E0521C5C
:102F7000BA42F0D3A5B19CF80110491CC9B28CF833
:102F8000011032290ED9CA4A8CF801E001211160E2
:102F9000C3B2E2B2C4F30721ED2002F081FC01E0EC
:102FA0008CF801E028464BE6C24A10B51268044688
:102FB0000020128D891A0BB2BC49096806E034F969
:102FC00011209A4201DCDA4200D50120491EF6D2D6
:102FD00010BD70B5B74D024600242868C07B40077D
:102FE0001CD51046FFF7E0FF012817D1FDF73CFA8A
:102FF000B14C206840F002002060FDF733FA4FF436
:103000000041002003F044FD286822780121C07BA4
:10301000C0F38003072002F043FC0124204670BD6A
:1030200030B5A149A34B0022CD681B68002D144682
:103030004FEAC07505D07DB185070DD58D782DB1CE
:103040000AE04DB1850707D58C7005E001258D702C
:103050000C7193F89750CD7010B18C7834B901E0B1
:103060008C700C71024693F89700C870104630BD02
:1030700010B58D4CA078002805D0E07820B1401E16
:10308000E070207910B910BD012020718348032120
:103090005838007902F080FF0020A070207110BD28
:1030A000F0B5864C804F0E4620780025A8B1B6F9C1
:1030B0000600B7F90A100A1A00D552427D4910B22B
:1030C0000968B1F86010814207DA00207C4920705D
:1030D000022001250870FFF7F8FC387821780843B2
:1030E00001D1F08878812846F0BD2DE9F74F84B0F2
:1030F0004FF000086C4ECDF80480CDF80880CDF874
:103100000C8015464446B6F908100498FFF716FFE0
:1031100001282DD0B6F908100498FFF75AFF0128AE
:1031200034D0644F386890F83A00000704D55F48FF
:103130000168049800F003FADDE90401FFF73DFEA1
:10314000824601287ED003F0DBFF0128FAD05948DF
:10315000DFF870B1DFF870910068C07B01074F485D
:1031600000F1320022D55949097801291BD01DE010
:103170004F480068012808D170694FF00051401E87
:10318000706111F8360F03D00870002007B012E606
:1031900040F002000870887820F0020088704C49E6
:1031A00000200860FDE74B49097879B1C9F80000B3
:1031B000CBF800000022012311460095FFF752FDD5
:1031C000070022D04348007858B11EE0334FC9F8B9
:1031D0000070CBF8000000231A46194638460095C7
:1031E000ECE73846FFF72EFD0190042101A8FEF719
:1031F0003FF9C0B202460095039001230199DBF824
:103200000000FFF72FFD00EA07084046FFF71AFD10
:103210000290042102A8FEF72BF900F0FF082D48C8
:1032200020490078097808437ED1224F386890F809
:103230003A00000710D5F079A8420DD0284600F0DA
:103240007BFF00E0B6E0284601F019F9284601F0BE
:103250001EFA284601F026FBB8F1000F58D00120D5
:10326000B8F1010F06D90D4900205039B1F803100B
:1032700001B10120F16879BB0028386890F83A0064
:103280004FEA007029D000282FDA002202A9D9F8CD
:10329000000000F0E4FB040027D033E044390120B3
:1032A000B05801205D0510008C02100014051000BC
:1032B0006805100054051000740510007A05100010
:1032C000800210002805100024051000F04F012096
:1032D0005C0900225C05100007E0002805DA02A95D
:1032E000D9F8000000F0A7FAD5E7386890F83A005E
:1032F00080070DD57D4802A90278D9F8000000F0BA
:103300002DFA0446012C03D1386890F85F00B071A3
:10331000029870B9386890F83A00000709D5294634
:10332000049800F022F900E020E010B101280AD052
:103330000CE05CB97079012808D1B07930B1401E39
:10334000B071F57136E00020B071044674713868D0
:1033500090F83A00400709D5029838B1B8F1010F4A
:1033600004D102A9DBF8000000F08CFEF571032205
:10337000F168029800F088F804460499FFF790FE7F
:103380005B4DC8B100246C6020464246059B039902
:1033900002F0B6FA2879214602F0FEFD4FF0010A4C
:1033A00054480078042803D002990498FFF787FC5A
:1033B0006868F0605046E9E6686884420ED0E0B282
:1033C0006C60FFF72DFE044628794246059B039961
:1033D00002F096FA2879214602F0DEFDFFF748FE5A
:1033E000DEE72DE9FF4F9146864600250D9F46E01A
:1033F00005FB07F00199012247F6FF7C01EB40062F
:103400006FEA0C040EEB400B13460021C9F1000AD1
:1034100016E036F9110048450FDA50450DDD8445B8
:1034200000DD8446844200DA0446002802DA4FF0C8
:10343000000202E001DD4FF0000301F1010189B259
:10344000B942E6D352EA030009D012B1012A04D0EE
:1034500004E0012B02D1204601E023B1002041000D
:103460000BD0002107E06046F9E736F81120121A68
:103470002BF81120491CB942F7DB6D1CADB2039843
:103480008542B5D3BDE8FF8F2DE9F043DFF86880B2
:1034900004461748D8F81010184B84EA010C144F52
:1034A000002140684FF001090D371E6812E009FA4B
:1034B00001F313EA0C0F07D0234202D096F83B50D9
:1034C00001E096F83E507D547D564DB16D1E7D5401
:1034D000491C09B29142EADBC8F81040BDE8F0830C
:1034E000234201D01843F3E79843F1E71405100095
:1034F000EC380120700210008C02100054051000FE
:10350000F0B588496425884E096811F86C2F497810
:103510004A43D3B2002202FB03F106EB410400212F
:1035200004E030F8117024F81170491C9942F8DB5E
:10353000521CAA42EFDB7D4900204870F0BD0B46CB
:1035400030B47A4904464878401CC0B248706428B8
:1035500001D9002048705A00C0B27349584301EBAA
:103560004000214630BC03F06ABC2DE9F34F70A047
:103570008B46ADB007C829AB4FF0000A83E80700BF
:10358000DFF8A8916D4EDFF89C815446554629A876
:10359000415D99F80100401A6421643090FBF1F21A
:1035A00001FB1200C7B2342101A803F0E9FC306826
:1035B0005D494200784301EB40010EA803F03FFC57
:1035C000022003F016FB308800B200905C4890F9AE
:1035D00000300EAA01A82D9902F059FB022003F039
:1035E00023FBD8F800004746C07B000714D5554898
:1035F0000078012810D15448007868B95348007801
:1036000050B1308801A900B20090514802680846C4
:10361000938E243202F0DFF9306801A942001BA822
:1036200003F052FC3278012301A91BA8FFF787FBA6
:103630004849002001ABD6F800C005E033F910205E
:103640008A4200DD1146401C6045F7D33868B0F867
:10365000620088422FDC0022012311461BA8CDF80E
:1036600000B0FFF7FFFAFFF7EDFA0746C00708D0F2
:1036700001200246289028A901A800F0F0F900B91D
:103680000124B80709D50220289034B9012228A9BD
:1036900001A800F0E4F900B90124780702D504205C
:1036A000289014B1012C0CD005E0012228A901A812
:1036B00000F0D5F928B1ED1C092DFFF668AF4CB329
:1036C0002BE0D8F800101948444691F8642001789E
:1036D000491CC9B2017091421FD90021017002201A
:1036E00003F087FA30680EA942001B4803F0A7FBDD
:1036F000022003F099FA20681722012190F8B10006
:1037000000F00103052002F0CBF8FEF7B5FF4FF003
:10371000010A02E0002089F800002FB05046BDE801
:10372000F08F000054051000DA390120A4021000C7
:103730000204070A0F142846630000001405100055
:103740006C051000F04F01205C0510007905100099
:10375000580510000080FFFFB058012010B5086820
:103760000024072802D1002001240860FE480068D8
:1037700090F8E307DC2804D11CB17F22114601F048
:103780008EFF204610BD2DE9F04708AC002594E8D7
:103790000016FF242E462F4609E033F9168088458F
:1037A00004DB16F0FF0404D1076033E0761C6645A5
:1037B000F3DB066876B3FF2C2CD003EB440636F916
:1037C000026C8E4228DC33F91480884524DB09EB37
:1037D000440339F914C033F9023C891BACEB030CE8
:1037E0000CFB01FCA8EB06069CFBF6FC63443AF9D3
:1037F00014C00AEB44041BB234F9024CACEB040CC9
:103800000CFB01FC9CFBF6F1214409B28A4201DB6E
:103810009A4201DD012507602846BDE8F08770B5B2
:10382000DDE90545049E012D02D002600B6070BDEC
:1038300006600C6070BD2DE9FF5F0026054603960B
:10384000086804278846344606285BD1B5F9080085
:10385000002800DD0446B5F90A00002801DD2044F7
:1038600004B2B5F904002146002801DD084404B281
:10387000B5F90600002801DD204404B24FF47A7047
:10388000414391FBF4F00FFA80FBB5F902004FF4CD
:103890007A71484390FBF4F00FFA80FAB34852462D
:1038A000A0F10801CDE90010A0F1100302975946DC
:1038B0004046FFF768FF06004FF0000917D1B5F941
:1038C00000004FF47A71484390FBF4F00FFA80F94E
:1038D000A6484A461830A0F10801CDE90010A0F131
:1038E0001003029759464046FFF74DFF0646A04891
:1038F000A0F800B0A0F802A0A0F80490B8F800105A
:10390000C1800681D8F8000003284BD1B5F900002A
:10391000002800DD0446B5F90200002801DD20443E
:1039200004B2B5F904002146002801DD084404B2C0
:10393000B5F90600002801DD204404B24FF47A7086
:10394000414391FBF4F00FFA80F9B5F90A004FF406
:103950007A71484390FBF4F002B284480297303009
:10396000A0F10801CDE90010A0F11003494640463E
:10397000FFF709FF060015D1B5F908004FF47A7179
:10398000484390FBF4F002B2784802974830A0F127
:103990000801CDE90010A0F1100349464046FFF7A9
:1039A000F2FE0646D8F80000052846D1B5F9000019
:1039B000002800DD0446B5F90200002801DD20449E
:1039C00004B2B5F908102046002904DDA988EA8868
:1039D000014411440CB24FF47A71484390FBF4F067
:1039E0000FFA80F9B5F906000297484390FBF4F00E
:1039F00002B25E486030A0F10801CDE90010A0F1EC
:103A0000100349464046FFF7BEFE060015D1B5F942
:103A100004004FF47A71484390FBF4F002B253482B
:103A200002977830A0F10801CDE90010A0F1100351
:103A300049464046FFF7A7FE0646D8F8000050B9B1
:103A400049480126006890F8E307DD2803D10021EA
:103A5000039A01F024FE04B03046BDE8F09F2DE942
:103A6000F04F054687B040480024069400680426BD
:103A7000DFF8FCA090F8E39717468B46B9F1DC0F0E
:103A80001FD18C21504603F059FADBF80000C0F337
:103A90000741AAF800109BF80010AAF80210298824
:103AA000AAF804106988AAF80610A988AAF80810CC
:103AB000E988AAF80A102989AAF80C106989AAF8D5
:103AC0000E109BF80000C0077ED04FF00008B9F13F
:103AD000DC0F02D10B21AAF81410B5F90000002860
:103AE00000DD8046B5F90200002803DD00EB080187
:103AF0000FFA81F84FF47A71484390FBF8F00FFA0F
:103B000080F9B5F906000297484390FBF8F000B23F
:103B100005901848A0F10801CDE90010A0F1580364
:103B2000A0F1600203A904A8FFF779FEDDE9030113
:103B3000CDE900100F4B0296683B49465846059A5E
:103B4000FFF721FE04460848006890F8E307DC28E8
:103B500004D1AAF816900599AAF81810002C33D1B0
:103B6000B5F9040008E00000540510008E041000B0
:103B7000624D01200E0310004FF47A71484390FB10
:103B8000F8F004B2FE480297A0F10801CDE9001058
:103B9000A0F15003A0F1580203A904A8FFF73FFECB
:103BA000DDE90301CDE90010F54B2246603B0296AA
:103BB00049465846FFF7E7FD0446F248006890F88A
:103BC000E307DC2809D100E046E00C21AAF81E102A
:103BD000AAF820900599AAF82210ECBBB5F90A00C2
:103BE0004FF47A71484390FBF8F000B20590E44836
:103BF00002971030A0F10801CDE90010A0F14803B0
:103C0000A0F1500203A904A8FFF709FEDDE90301B2
:103C1000CDE90010DA4B0296483B49465846059AD2
:103C2000FFF7B1FD0446D748006890F8E307DC28A9
:103C300007D10D21AAF82810AAF82A900599AAF808
:103C40002C104CB9B5F908004FF47A71484390FB39
:103C5000F8F00FFA80F800E028E0C9480297203019
:103C6000A0F10801CDE90010A0F14003A0F1480245
:103C700003A904A8FFF7D3FDDDE90301CDE9001096
:103C8000BF4B4246303B029649465846FFF77BFD04
:103C90000446BC48006890F8E307DC2806D10E21F2
:103CA000AAF83210AAF83490AAF836809BF80000DF
:103CB00080077CD5B5F904004FF00009002800DD2D
:103CC0008146B5F90600002803DD00EB09010FFA73
:103CD00081F94FF47A71484390FBF9F000B20590F6
:103CE000B5F90200484390FBF9F004B2A44803A9D7
:103CF00088300090CDE90107A0F15003A0F15802EF
:103D000004A8FFF78CFDDDE90301CDE900109C4B11
:103D100022462833029658460599FFF734FD04469B
:103D20009848006890F8E307DC2807D11521AAF825
:103D30003C100599AAF83E10AAF84080002C36D114
:103D4000B5F900004FF47A71484390FBF9F00FFA8F
:103D500080F88B4802979830A0F10801CDE9001057
:103D6000A0F14803A0F1500203A904A8FFF757FDF2
:103D7000DDE90301CDE90010814B42464033029654
:103D800058460599FFF7FFFC04467E48006890F806
:103D9000E307DC2807D15046162120F8461F059975
:103DA0004180AAF84A8014B9B5F90A0000E064E03D
:103DB0004FF47A71484390FBF9F00FFA80F870489D
:103DC0000297A830A0F10801CDE90010A0F140034E
:103DD000A0F1480203A904A8FFF721FDDDE90301D2
:103DE000CDE90010664B4246583302965846059975
:103DF000FFF7C9FC04466348006890F8E307DC2835
:103E000007D15046172120F8501F05994180AAF884
:103E1000548094BBB5F908004FF47A71484390FB85
:103E2000F9F00FFA80F856480297B830A0F108016F
:103E3000CDE90010A0F13803A0F1400203A904A8C5
:103E4000FFF7EDFCDDE90301CDE900104C4B4246E4
:103E50007033029658460599FFF795FC0446494889
:103E6000006890F8E307DC2807D15046182120F8B5
:103E70005A1F05994180AAF85E809BF80000400710
:103E80007CD5B5F908004FF00008002800DD804619
:103E9000B5F90A00002803DD00EB08010FFA81F8EC
:103EA0004FF47A71484390FBF8F00FFA80F9B5F9B6
:103EB00002000297484390FBF8F000B205903248A8
:103EC000A0F10801CDE90010A0F15803A0F16002B3
:103ED00003A904A8FFF7A3FCDDE90301CDE9001065
:103EE000294B0296683B49465846059AFFF74BFC1A
:103EF00004462448006890F8E307DC2807D11F2116
:103F0000AAF86410AAF866900599AAF86810002C1F
:103F100034D1B5F900004FF47A71484390FBF8F0C2
:103F200000B20590184802971030A0F10801CDE9C1
:103F30000010A0F15003A0F1580203A904A8FFF754
:103F40006EFCDDE90301CDE900100F4B0296503BFA
:103F500049465846059AFFF716FC0446094800688A
:103F600090F8E307DC2805D12021AAF86E10059906
:103F7000AAF8701014B9B5F9060007E068E000006F
:103F80001E03100054051000460410004FF47A710F
:103F9000484390FBF8F000B20590FE480297A0F16C
:103FA0000801CDE90010A0F14803A0F1500203A9D7
:103FB00004A8FFF734FCDDE90301CDE90010F54B5F
:103FC0000296583B49465846059AFFF7DCFB0446E3
:103FD000F148006890F8E307DC2807D12121AAF80E
:103FE0007810AAF87A900599AAF87C1084BBB5F9E4
:103FF00004004FF47A71484390FBF8F005B2E548AD
:1040000002971030A0F10801CDE90010A0F14003A3
:10401000A0F1480203A904A8FFF701FCDDE90301B0
:10402000CDE90010DB4B2A46403B029649465846F4
:10403000FFF7A9FB0446D848006890F8E307DC289E
:1040400006D12221AAF88210AAF88490AAF88650F4
:10405000DBF8000050B9D0480124006890F8E3076D
:10406000DC280BD10021069A01F019FBCA48006830
:1040700090F8E307DC2801D1AAF8124007B02046E7
:10408000BDE8F08F2DE9F0418EB00C468046002649
:1040900035463421684602F073FFC04F41466846FA
:1040A0003A6801F03FFD397840F6FF7268462368B0
:1040B00000F09AFDBA49024620680B7820EA030313
:1040C000DF07B54B09D01F68B7F84F70974204DD82
:1040D00020F0010001252E46206087070CD50F78BF
:1040E000BF0709D41F68B7F85570974204DA20F06B
:1040F00002000126AD1C2060470710D5097849074A
:104100000DD41968B1F85770974203DCB1F8591013
:10411000914204DA20F0040001262D1D2060186869
:1041200090F8E307DB2803D12946FD2001F0A0FA2F
:104130000EB03046BDE8F0812DE9F04FDFF8648223
:104140004FF42F7208F10805DFF85CC24FF0A00AA7
:104150004FF4A57B4FF47A7340F2924E4FF41676EB
:104160006FF01D0405F10807C2F1000905F1100107
:1041700000287DD001287CD002287BD14FF0DC0ABA
:104180004046A8F800A0468046464FF44870B080EC
:1041900030461036C38040F27A3028804FF4CD701C
:1041A00068804FF49670A880A1F110006425C58046
:1041B0005A20388038464FF4E177A0F802C04FF615
:1041C0000C60B080A6F80690FA2608460E8047805C
:1041D00040F28A2CA0F804C040F25230C8807249E4
:1041E00008F120005A31018008F120084FF6F260F2
:1041F000A8F80200A8F804004FF65C60A8F80600D2
:1042000008F108084FF6E040A8F800006748A8F851
:104210000200A8F804004FF69040A8F8060008F144
:10422000080006804780A0F804C0C38008300580DD
:104230007825458096258580B425C5800830018085
:104240004FF6E8614180714281806FF0DB01C180EF
:1042500008304FF4C871A0F800A041808280C3806C
:10426000083014210180418028218180322102E020
:104270000BE07AE008E0C1806100083001804180F5
:104280006FF027018180C480FAE6A8F800A0DFF86B
:1042900014814046A8F802B08280C380A5F800E0EF
:1042A00008F1080540F22A306880284686804FF4DD
:1042B000FA70E88005F108003C80A0F802C03B4895
:1042C00005F108048230A080A4F80690A0200880A0
:1042D00005F110004FF4C87444808280C380083018
:1042E0004FF6A26101806FF0630141804B10838023
:1042F0006FF09501C18005F120012D4808804880AC
:104300008880C88005F12800B42101804480828023
:104310004FF46171C180083003805A2343806423C5
:1043200083807823C38008304FF63E6303804FF6C6
:10433000CA6343804FF6D46383804FF6E863C3803B
:1043400008309623038044808280C1802821083071
:1043500050220180462141808280C18008306FF068
:104360009F0101806FF0810183E0A8F800A0DFF8D1
:1043700034804046A8F802B08280C380A5F800E0EF
:1043800008F1080540F22A306880284686804FF4FC
:10439000FA700FE0660410005405100014051000B8
:1043A00098021000A60210007AFEFFFF26FDFFFF14
:1043B00082FBFFFFE8803C8005F1080005F108045E
:1043C000A0F802C0FC48A080A4F80690A1F800A0C4
:1043D0004FF4C8744C808A80CB8005F118004FF6EA
:1043E000A26101806FF0630141806FF081018180E3
:1043F0006FF09503C38008304FF6823303804FF689
:104400007C4343804FF65E4383804FF64A43C3802C
:104410000830B4230380448082804FF46173C380EA
:1044200008306FF0310505805A2545806425858068
:104430007825C58008304FF63E6505804FF6CA6581
:1044400045804FF6D46585804FF6E865C580083015
:104450009625058044808280C3800830282202800F
:104460004622428050238380C28008306FF09F0232
:10447000028041806FF077028280C18000E62DE9E2
:10448000F04FCE4A00214FF4167640F2DE3C4FF456
:104490007A734FF0B40B02F108044FF0E60E6FF0A0
:1044A000DB0902F110056FF0A90A6FF0950702F120
:1044B0001808002877D0012875D0022871D1118002
:1044C000104672104680A0F804C0C38021462280A6
:1044D000234696204880642199804FF4E171D98069
:1044E000B54C083364342C804FF6765159804FF622
:1044F000445199804FF61251D9800021A8F800103C
:1045000008334FF448715980414640F2B6338B80EE
:1045100008354FF47A71E98008F108014FF44875C5
:104520000D8048808A80CD80083100250D804FF6AF
:104530003E654D808C804FF6A854CC800831002415
:104540000C804FF448744C808B804FF47A74CC808C
:10455000083132240C804880AA248C80CA8008311B
:104560006FF0F9020A804A806FF0E5028A804FF608
:10457000D462CA80002208310A804E808B804FF4BA
:104580007A72CA800831822208804A8046228A8054
:10459000C88001F108006FF08101078041808180AF
:1045A000C7806DE5FFE711805680A2F804C0D38074
:1045B000A4F800B0A4F802E0FA20A08040F2622043
:1045C000E080A5F800907C48A5F802A0AF80D2302A
:1045D000E8807A48794C1830A8F8001040F2262577
:1045E0004580183440F2DE30A0802046B424C380D9
:1045F0000830524604804FF4AA74448064008480DA
:1046000040F21454C48008306FF0DB0404806FF073
:104610003B044480502484806FF06304C4800830DD
:104620000180458040F2DE358580C3800830462514
:104630000580651045808480C28008306FF0E504F5
:1046400004804FF6A26444804FF6706484804FF675
:104650002A64C48008304FF416740180448040F20C
:10466000DE348480C3800830322303801E234380DD
:1046700081800A21C18008306FF06D0101806FF0E8
:10468000810141806FF09F018180C280F8E42DE9B3
:10469000F04FDFF82881282508F1980832224623B8
:1046A0006FF063064FF4C87740F2EE2C4FF47A793E
:1046B00008F1080A08F1100B08F118014FF0FA0E82
:1046C0004FF4167400287BD0012879D0022871D1CC
:1046D0006420A8F800004FF4AF70A8F8020040462C
:1046E00084801001A8F806005046AAF800604380B4
:1046F000534682209880D8804FF67063ABF8003024
:104700005B466FF0E50058806FF0A9009880D88074
:10471000642008804F808C80A1F806C003F110004F
:10472000711001804280502181806421C180083055
:104730006FF0F90101806FF0950141806FF0770310
:104740008380C68008306310028043804FF42F734B
:104750008380A0F806900830058042808280C58062
:1047600008306FF09F02028041808180C280083053
:104770006421018047804FF4FA71818040F2DA2190
:10478000C180083040F2E241018040F28A2141803C
:104790004FF4D27181804FF42A71C18008304FF6F6
:1047A000A261A0F800E041804FF6BC5181804FF635
:1047B000F851C18064E403E0A8FDFFFF4603100048
:1047C000FF48A8F8006006464780A0F804C0A6F895
:1047D0000690AAF8005006F108053C20688028469B
:1047E00082802A463220D0806FF06302ABF800202E
:1047F00005F108026FF04F0050806FF05900908073
:10480000D0806FF06300088002F108010846A1F82B
:1048100002E084804FF47A70C88001F10800103102
:10482000038043808380C3806FF0810008804880CC
:104830008880C88008316FF063020A804FF4967256
:104840004A804FF42F728A804FF47A72CA800831FE
:1048500014220A801E234B808B80CA8008316FF09F
:104860008B020A8048808880CA8005F140006FF082
:1048700063010180DC21418084804FF47A71C18022
:104880003221083001809621418081806421C180DD
:1048900008304FF612510180CA49418081804FF69D
:1048A000445186E72DE9F04FDFF814C300210CF1E5
:1048B000A00C0CF10804142332274FF0500A4FF4D7
:1048C000167640F2B6386FF0270B04F108096FF046
:1048D0001D026FF0090E04F1100500287DD001289B
:1048E0007CD002287BD16420ACF800004FF4AF707C
:1048F000ACF802006046C84686804FF42F70ACF8D2
:1049000006002780A5F110075A247C806424BC800F
:104910008224FC806FF0F907A9F800704C466FF014
:10492000D10CA4F802C06FF0C707A7806FF0A904EC
:10493000A8F806404FF48278A5F8008009F108082D
:104940004FF4E175A8F80250A8F804604646F080DC
:1049500008F10800BE260680C8264680FA26868012
:104960004FF49676C68008306FF09506A0F800C028
:10497000478086807E10C68008304FF4C877078055
:1049800040F22627478040F28A2787804FF44877F5
:10499000C78008301E2702800A2242808780642751
:1049A000C78008306FF0E50707806FF0BD074780CC
:1049B0008480C680083040F276240580448040F22E
:1049C000DA24848040F26634C4800830018042805A
:1049D0008380C2800830068002E00AE077E002E1CE
:1049E0006FF0590141806FF03B0181806FF045010C
:1049F000F8E07348ACF800A0A030DFF8C4C14680EE
:104A00000CF1A00C40F28A20ACF804006046A0F83B
:104A10000680238008300CF1080347801E20988010
:104A20002820D88003F10800A9F800B0428008339C
:104A30007046A3F804E0D9801421298008334FF48C
:104A4000E171598040F2EE21998040F2B631D9806F
:104A50000CF120014FF491730B804FF4C3734B8022
:104A60004FF4AF738B804FF4A573CB8008316E2366
:104A70000B8048808880CA8008314FF4FA750D8019
:104A800040F202334B8040F252338B804FF461741A
:104A9000CC8008316FF081030B806FF063074F808B
:104AA0006FF06D078F80CB8008316FF0BD030B80F6
:104AB0006FF0C7074F808B806FF0E503CB80083124
:104AC0004FF42F730D804E808B80CC8075E0ACF856
:104AD00000A0DFF8ECC03A480CF1A00C4FF4AF7A1C
:104AE000ACF802A0A0304FF4617CA0F804C0A0F89C
:104AF000068023800830324B4780A8333C209880C2
:104B00002820D88003F10800A9F800B042800833BB
:104B10006FF02700988018464FF4FA74C180142073
:104B2000288003F108004FF4E171418003F108018E
:104B300040F2EE20888040F2B630C88003F11000C9
:104B40004FF4917101804FF4C3714180A0F804A02B
:104B50004FF4A571C18003F118016E200880A1F8FF
:104B600002E0A1F804E0CA80083140F202330C8070
:104B70004B8040F252338B80A1F806C008316FF0B1
:104B800081030B806FF063054D806FF06D058D80A4
:104B9000CB8008316FF0BD030B806FF0C7054D80EF
:104BA0008B8070466FF0E503CB8008314FF42F7394
:104BB0000C804E808B80A1F806C00149F03103E0E3
:104BC000DE03100076FDFFFF0A80488088806FF0CA
:104BD0001300C8801B486FF045010180418081802F
:104BE0006FF03B01C18049E42DE9F0410024491EEA
:104BF00017468646CAB2A44626462546D80701D09F
:104C000002220DE098070BD50124032208E03EF9AB
:104C10001400604502DD00FB04660544641CE4B238
:104C20009442F4D985FB012386FB070102F0E3F8E7
:104C3000002800DA0020791E884200DD084600B214
:104C4000BDE8F081D60410004749096891F9242194
:104C5000824201DA0120704791F91C11814201DD85
:104C60000220704700207047404908B50020C86006
:104C70008860012248600A703D4A142111703D4944
:104C800008600871FDF7FCFEFDF7C6FBFDF7F8FCB8
:104C9000FDF74EFF6B4600220121022001F048FF84
:104CA0000098C007F6D00121022001F020FF00F09B
:104CB00001F8EFE7F8B50027032001F09AFF00F0B4
:104CC0002EF82A4C2A4D2C4E207BC0070BD095F98C
:104CD0000000FFF7B9FF307095F900100246206917
:104CE000FEF703FA0746A06870B1022001F081FFC9
:104CF0003078009095F90030D4E90412A068FDF7EF
:104D00003FFC022001F090FF012F03D11B492069D5
:104D1000FDF760FEBDE8F840032001F085BF70B5E7
:104D2000124C174DE068B5F90C1080EA0102D20769
:104D300008D0C90702D0FDF7A3FE03E0C00701D0E9
:104D4000FDF70BFFB5F90C00E0602869A060A868CA
:104D500060600B481630206128782070287D6070D4
:104D60000848606170BD0000540510001005100077
:104D70006C051000F43801207C0510008002100042
:104D80002807100044390120094C00202060401CF5
:104D90002060FBF730FD00F0B9FEFBF7FFFB08B920
:104DA000FCF7E5FBFBF744FA01F062FC2068EEE754
:104DB0002C051000F74900200860F7490860F74902
:104DC0000860F74908707047D0214DF6C062BA20DC
:104DD00000F07CBC70B54FF40063984202D2F14CF5
:104DE000246807E0A0F5805080B24FF480539842C9
:104DF0000CD2ED4C85189D4200DD1A1A002303E009
:104E0000CD5C1E185B1CA5559342F9DB70BDB0F557
:104E1000805F04D20A460146E248006808E0B0F527
:104E2000FE5F07D3A0F5FE5080B20A460146DE4879
:104E300000F069BC704701F04CB810B54FF4005158
:104E4000002000F0D3F90023BDE810401A461946AF
:104E5000032000F025BD10B54FF48041002000F084
:104E6000C5F90023BDE810401A461946042000F099
:104E700017BDC8490A6882430A600221012000F078
:104E8000B5B9C4490A6802430A600221012000F052
:104E9000ADB9FBF74CBEFBF725BE10B5C00711D06E
:104EA000C24800230222016841F001010160012192
:104EB000052000F0F5FCBDE810404FF40061002033
:104EC00000F094B910BD10B50324FBF7CDFAB84833
:104ED0000460FBF7C7FA002301211A46084600F0D8
:104EE000DFFCBDE810404FF40031002000F07EB937
:104EF00010B5002301221946104600F0D1FCBDE890
:104F000010404FF48051002000F070B910B50978BE
:104F1000A8480024012908D0047040F67101A64871
:104F200002F00CF8A548048010BD01210170F4E7DF
:104F30000421012000F05AB99A4A10B512680446BB
:104F40009F4892F8E327012C02D0022C05D006E0FE
:104F5000882A10D00978017001E0882A02D0892AB5
:104F600003D008E04978017005E0017800231A4673
:104F7000172000F095FC8A480178002903D1002C05
:104F800001DD0121017010BD844A00230128136056
:104F900005D1087810211060012000F027B9704772
:104FA0004FF48021002000F021B94FF400210020AF
:104FB00000F01CB97B480021006890F86800C00729
:104FC00011D080480068827A12B1FF2A03D00AE02B
:104FD000C27A1AB107E0C27AFF2A04D196218172FF
:104FE000A521C172012100231A46102000F058BCEF
:104FF000744800210B4600680A468172C172202065
:1050000000F04EBC00280DD008786F4A01280AD065
:1050100002280BD003280CD0042803D1B1F80100DA
:10502000A2F80300704748781070704748785070B5
:10503000704748789070704710B50978634C00202D
:1050400031B10121217062490870FDF73EFD00E099
:1050500020700120FFF721FF00232178BDE81040D8
:105060001A469A2000F01CBC10B5584C2278D2B9D0
:10507000574A1278BAB1574A042809D00020107054
:10508000002321781A469F20BDE8104000F008BC9C
:10509000514B0888188048885049088001201070BA
:1050A000FDF713FDECE7474A00EBD070136820F0E2
:1050B000010203F1340001F0C2FE00231A462178F8
:1050C0009C20E1E7414A1278002A0BD0012809DC34
:1050D0003C480978002300681A4680F83A109D2061
:1050E00000F0DEBB704770B5384C2278A2B1354D68
:1050F00000EBD07626F001022B6803F1240001F0CA
:105100009EFE29687008002348842178BDE870401D
:105110001A469B2000F0C4BB2D480078002811D10E
:10512000204B2F4A2F4C1B6808E031F8105022F812
:10513000105031F8105024F81050401C93F86C5067
:105140008542F2DC70BD70B51E4A4D78431E14686E
:105150000A781D445434202D02DBDBB2FF2108E025
:10516000A318421E1846491C01F069FE00231A4686
:105170000121BDE87040992000F092BB30B41A4C78
:1051800000B1087820700023C1B230BC1A46A320B9
:1051900000F086BB60051000640510006805100073
:1051A0007B05100054051000500001207005100010
:1051B000740510003C051000F24F0120340510006A
:1051C0006C05100058051000F43801205C05100033
:1051D000F04F012078051000EC380120EE38012056
:1051E000B0061000BA0610005D05100038B50C4678
:1051F000054601F04DFC6946284601F088FC009AFE
:105200002242F8D138BD000010B52021634801F0DA
:1052100095FE6248FBF792FC6049401E11F8012B95
:10522000A2F190031F2B01D85D4A05E0A2F1C00353
:105230000F2B06D85A4A803252F82320BDE810407E
:105240001047B82A21D00DDCB02A13D0B22A27D1BA
:10525000032825D108888A78BDE8104040BA114655
:10526000FFF7D5BDFB2A17D0FC2A19D1BDE81040A5
:10527000FFF7F1BD022813DD31F8022BBDE8104025
:1052800053BA821E1846FFF7A5BD022808D1088828
:10529000BDE81040FFF7CFBDBDE81040FFF7CDBD22
:1052A00010BD0120FFF7EDBD0120FFF7E2BD10B5F5
:1052B000FDF7E6F9BDE810400120FFF7EEBD00F074
:1052C0006ABA384810B5017800290CD00221017063
:1052D00035480068002806D0FDF7D2F9BDE8104037
:1052E0000120FFF7DABD10BD2E480178002903D058
:1052F00003210170FDF7E9BB704770B52B4D2C4CB5
:105300000020287020680078A52802D0012000F035
:10531000CFF840F2FF112068FCF790F82168D1F82F
:10532000FC17814202D0022000F0C2F840F2FF31A7
:105330002048FCF783F81F49D1F8FC1F814206D0B2
:1053400020680079800702D4032000F0B1F81A48E1
:10535000007881074FF0010001D5287070BD114918
:105360000870FDF7B2FB0120FFF797FDBDE8704024
:105370001248FEF7C5B80B4910B500200870FDF7BC
:10538000A4FB0B480068007A800701D5FFF7D0FD29
:10539000BDE810400120FFF780BD0000C4061000EA
:1053A0005475000079051000980210007A0510006D
:1053B0005405100050000120F0380120B0580120A1
:1053C00008B5FFF7F7FC00F0C9F91B4C206800791D
:1053D000800701D5FFF777FD20680079C00701D06D
:1053E000FFF75FFF2168C87B00070DD511F86C0F30
:1053F0004978484300F0BAFA104900231A46087069
:105400000146C02000F04CFAFDF75FFB01216B461E
:105410000022032001F08CFB0098C007F6D0FFF7B4
:10542000F3FE0121032001F062FBFBF79BFBEDE79C
:105430000121032001F02CBB54051000F04F012086
:10544000304C2F4AC4E900210168A1604168E16045
:1054500081682161C16861610169A1614169E1619E
:1054600081692162C069606204F12800FCF78FF84D
:1054700001F077FC606400F035F82249224AC1E966
:105480000020704710B501284FF0000205D00146FA
:10549000BDE81040022000F019B90121022000F0FF
:1054A00015F900F01FF8012801D10220EAE7704742
:1054B00010B5044601460022032000F007F9012C34
:1054C00001D0022C01D100F00DF810BD00220146E0
:1054D000062000F0FBB801460022072000F0F6F895
:1054E00000F000F8FBF787F94FF0005010F8361F76
:1054F00041F002010170817821F002018170FEE724
:10550000AF0550FA00EE0120BA0110AB77B585B0B7
:105510000E46BDF814401546200A40EA0420ADF8B6
:1055200014004F48BDF8141000240180A0F58070CD
:10553000CDE900044B480294039400681346484A9E
:10554000C0790221FBF77BFA08B02A463046BDE855
:105550007040454901F073BC17B581B00B46BDF8EA
:1055600004001446010A41EA0020ADF804003C485A
:10557000BDF8041020F8021B194601F060FC002061
:10558000009038480023364A0068A11CC079FBF718
:1055900025FA1FBD77B585B00E46BDF814401546F7
:1055A000200A40EA0420ADF814002D48BDF814107C
:1055B000002401802C48CDE900042A480294039479
:1055C00000681346264AC0790221FBF738FA08B072
:1055D0002A463046BDE87040234901F030BCFAF756
:1055E000EDBF08B50020ADF8000002226946FFF7C4
:1055F0008DFFBDF8000008BD00B587B00022012175
:105600000720FBF701FB072001F068FD00204FF4A5
:10561000FA7100BF401C8842FBDB072001F067FDE8
:10562000FFF7DFFFA0F584410E3902D00120FFF71C
:1056300029FFAFF2DB000190AFF22F100090AFF224
:10564000AB000290AFF2690003900848049040F26A
:105650008F20ADF814006846FBF776FB07B000BD5D
:10566000F04E012054051000F04D01205F050000B0
:105670001CB5DB238DF800308DF801008DF8021089
:10568000100E8DF80300100C8DF80400100A8DF830
:1056900005008DF80620684600F055F91CBD1CB5C4
:1056A000DB238DF800308DF801008DF80210100E0C
:1056B0008DF80300100C8DF80400100A8DF8050019
:1056C0008DF806206846FBF75CFA1CBD1CB50F235D
:1056D0008DF800308DF801008DF80210080A8DF861
:1056E00003008DF80420100A8DF80500100C8DF8C9
:1056F0000600100E9A498DF80700012008706846D0
:10570000FBF73FFA1CBD2DE9FC4100270646009738
:10571000122015460C4601978DF800001AE0200A69
:105720008DF80100C4F30B008DF80240315C304469
:105730008DF8031041788DF8041081788DF80510EC
:10574000C0788DF806008DF80770684600F0FBF809
:10575000241D2D1F002DE2DCBDE8FC811CB50020BE
:10576000804900900190096810234A7889788DF863
:1057700000308DF804008DF801008DF805208DF8BB
:1057800002008DF806108DF803008DF807006846BA
:1057900000F0D9F81CBD70B588B000240094142026
:1057A00001948DF80000FBF713FF8DF80100F22043
:1057B0008DF803006B4E37208DF804003068684D7B
:1057C00041788DF8051080788DF8060028788001E2
:1057D0008DF80700684600F0B6F800941520019493
:1057E0008DF80000306890F8EC178DF8011090F8F3
:1057F000ED178DF8021090F8EE178DF8031090F861
:10580000EF078DF80400287880018DF807006846BE
:1058100000F099F8009402A80194FBF7EAFD1B2020
:105820008DF800000298000E8DF801000298000C1F
:105830008DF802000298000A8DF8030002988DF896
:1058400004008DF8054004988DF806002878800142
:105850008DF80700684600F076F800941C208DF85B
:10586000000003980194000E8DF801000398000CCD
:105870008DF802000398000A8DF8030003988DF854
:10588000040005988DF8050006988DF80600287824
:1058900080018DF80700684600F055F808B070BD2B
:1058A0001CB5304C246894F8E247A40710D50024B6
:1058B0000194009416248DF800408DF801008DF8B5
:1058C00002108DF803208DF80430684600F03BF894
:1058D0001CBD1CB5002300930193E1238DF800301B
:1058E0008DF80100080A8DF80200100A8DF80400F6
:1058F0008DF803108DF80520684600F024F81CBDD3
:105900007CB5184C246894F89340E4071AD000241E
:1059100000940E258DF800508DF8010012488DF886
:10592000021001948DF80320B0F80300010A8DF8ED
:1059300004108DF805008DF806308DF80740684694
:1059400000F001F87CBD10B50446012001F051F9CA
:105950002046FBF716F9BDE81040012001F064B9BC
:105960003005100054051000F4380120F0B523492B
:10597000074601200A68518C59B32149096891F8FA
:10598000693092F83A108B4202D009B1FF2920D138
:1059900002F1340602F12404B51C00214FF6FF7C0D
:1059A000383208E034F811300BB1634501D10020E2
:1059B00003E0491C89B2B942F4D3318809B1FF2907
:1059C00000D10020298821B1FF2902D012889142FC
:1059D00000D20020F0BDF0B50024059E0AE031F9A8
:1059E000145032F814705D4395FBF7F520F814500D
:1059F000641CA4B2B442F2DBF0BD000058051000F4
:105A00005405100070B54E21324801F097FA314C20
:105A1000A620314D20804FF23720608028684178E1
:105A2000217180786071FBF7CFFDE080FFF7D9FD31
:105A30002081286890F86C10217790F86D106177BC
:105A40002649E18326492184264961842649A18784
:105A50002649A1842649E18426492185D0F8FC17EE
:105A60000A0C6285A185B0F83F10E185B0F84110BD
:105A70002186B0F843106186B0F84510A18690F8F1
:105A8000741001F0030284F83620C1F3011184F888
:105A9000371090F8681001F0010121871649096854
:105AA0004A8952BA628701F12202E2873232A4F8AF
:105AB000422090F8690004F8440F91F83A006070B1
:105AC0000E4824F8020F0E4860800E48A0800E4851
:105AD000E08070BD000001205405100064580120D2
:105AE000123901204439012076390120B0580120B3
:105AF000C4000120F038012058051000EC380120C6
:105B0000EE380120F4380120F24F012010B5FAF7E9
:105B1000ABFCFBF71AFD08B1FBF711FDBDE8104027
:105B2000FAF7A0BC30B501230CE000EB430531F8D7
:105B3000134025F8024C01EB430434F8024C20F8E2
:105B400013409B1C9342F0D330BD10B5FAF78CFC88
:105B5000FBF7FBFC08B9FBF7ECFCBDE81040FAF7DB
:105B600081BC2DE9F041BC4D0F465E00298890466E
:105B700001EBC10149000CB26968324601EB4403F4
:105B80000146184601F05BF96868324600EB4400B4
:105B900039460C3001F053F96868324600EB440096
:105BA0004146183001F04BF92888401C00B21E21F4
:105BB00090FBF1F201FB1201288029B9002807D0DF
:105BC000A6490A88521C0A803C2801DB0020288054
:105BD000BDE8F081F0B5851ADDE905471E1B754368
:105BE0008E1A012F02D0904206DD0BE0904201DCBC
:105BF0001846F0BD884201DB2046F0BD95FBF6F06B
:105C0000181AF0BD8842F3DA95FBF6F02044F0BD97
:105C10002DE9FC4F044692480B460026076835469E
:105C200007F58A7207F58E7C125707F5927807F50B
:105C3000967107F59A7907F59E7A07F5A27B1846C3
:105C400007F5A6779A4200DD10460957994200DA17
:105C5000084682420ADC1CF90430834206DB1946FE
:105C600019F9043001251AF9044008E018F9042054
:105C7000824209DC814207DB3B571BF90440CDE936
:105C80000045FFF7A7FF46B23046BDE8FC8F2DE97F
:105C9000F84F894672490546DFF8C8A108689B4657
:105CA000904690F8E307882808D12A68CAF80020AF
:105CB0006A68CAF80420AA68CAF8082000245AE0D2
:105CC000694839F81410664B076838F81400012643
:105CD000081A25F814001868243790F8E317882963
:105CE00006D139F8142038F81410511A2AF8141073
:105CF000C07BC0063DD55D480078D0BB5C480078CD
:105D0000012836D15B48007898B3A0B25946FFF716
:105D10007FFF01465248006890F8E307882805D1C4
:105D2000554880F830B2204480F831120AEB440024
:105D30008181F1B135F9140064225043C1F164024C
:105D400090FBF2F000B2002802DA0026404200B2D6
:105D500037F81420824205DC821A4A43642192FB00
:105D6000F1F1401A25F814001EB980B2404225F81E
:105D70001400641C24B20A988442A1DB38480068ED
:105D800090F8E307882835D12968CAF8181069689F
:105D9000CAF81C10A968CAF82010062000903248E2
:105DA00030490268183101F10C00938E2432FFF75C
:105DB00012FE314F284E6FF0130570883D54401C81
:105DC00070800024A0B22946FFF722FF7188641C6E
:105DD00024B27854491C7180062CF3DB6D1C6DB223
:105DE0003C2DEADB7088B0F50C7F07F800B001D3DA
:105DF00000207080BDE8F88F70B5002408E031F80D
:105E0000145032F81460AD1B20F81450641C24B2F6
:105E10009C42F4DB70BDF0B4049C012C04D01BB197
:105E2000C3F11006002412E0F0BC520001F007B8E4
:105E300030F9145031F914705D4307FB0655EF1724
:105E400005EB17752D1120F81450641C24B29442F0
:105E5000EEDBF0BC7047000034051000F24F01206B
:105E6000540510001A5B0120580510005C05100055
:105E7000F04F012079051000E25801200FB42DE900
:105E8000F05F0025DDF874A08B4681462E464FF06A
:105E9000010808FA06F7002407EA0B076FB108FAB1
:105EA00004F010EA090F08D0324621460C9800F0A1
:105EB000D1FA0AF805006D1CEDB2641CE4B2052CA1
:105EC000ECD3761CF6B2052EE3D3BDE8F01F5DF8E7
:105ED00014FB10B5044650212B4801F02FF82B4A33
:105EE0001178491C1170A00504D5BDE81040264862
:105EF00000F001B810BD2DE9F041044690B0A52096
:105F000020704FF40070A4F8010000F0AAF920718D
:105F100000F0A2F9607100F09AF9804600F092F961
:105F200005461B4800680179552904D1D0F80500C1
:105F300020F07F40A060174E392206F1740796F8D2
:105F4000B000207304F130000F90391D684600F056
:105F5000BBFF002229464046736FFFF78FFF04F115
:105F600010000F903922391D684600F0ADFF012264
:105F700029464046736FFFF781FF04480078E070C0
:105F800010B0BDE8F0810000008001203D05100048
:105F9000580510005000012070B52D4E05460C46E6
:105FA000306890F8940001070AD5E10700F0070077
:105FB0004FF0000201D0012100E00021FAF724FE99
:105FC000306890F8941008060AD5A007C1F30210B3
:105FD0004FF0000201D5012100E00021FAF714FE84
:105FE000306890F8950001070AD5690700F00700AE
:105FF0004FF0000201D5012100E00021FAF704FE74
:10600000306890F89610080712D51248007878B1D9
:106010001148007860B91148007848B910480078F4
:1060200000284FEA847008D0002810D1A8070ED1AC
:1060300001F007000022114605E00028F6D001F02B
:10604000070000220121BDE87040FAF7DDBD70BDF8
:1060500054051000790510005C0510005D05100066
:106060009002100010B5574C206890F8940001077A
:106070001CD500F0070001F03AF8206890F8940071
:1060800000F0070001F02AF820680022114690F87D
:10609000940000F00700FAF7B7FD206800221146CF
:1060A00090F8940000F00700FAF7C4FD206890F81B
:1060B000940001061CD5C0F3021001F018F8206806
:1060C00090F89400C0F3021001F008F82068002254
:1060D000114690F89400C0F30210FAF795FD20687D
:1060E0000022114690F89400C0F30210FAF7A2FDC6
:1060F000206890F8950001071CD500F0070000F01B
:10610000F6FF206890F8950000F0070000F0E6FF29
:1061100020680022114690F8950000F00700FAF779
:1061200073FD20680022114690F8950000F00700EA
:10613000FAF780FD206890F8950001061CD5C0F3A1
:10614000021000F0D4FF206890F89500C0F3021010
:1061500000F0C4FF20680022114690F89500C0F3BB
:106160000210FAF751FD20680022114690F89500C0
:10617000C0F30210FAF75EFD206890F89600010760
:106180001ED500F0070000F0B2FF206890F89600DE
:1061900000F0070000F0A2FF20680022114690F8EE
:1061A000960000F00700FAF72FFD20680022114644
:1061B00090F89600BDE8104000F00700FAF73ABDED
:1061C00010BD00005405100010B500F001F91B4986
:1061D0000020086010BD10B5FFF74FF9BDE8104072
:1061E000FAF7A5BC002101604160704710B5017944
:1061F00099B1134900220A604A608A60CA600F4957
:10620000D0E90020C1E90120081D00F01FF90B486A
:10621000001D00F0B3F9012010BD002010BD10B525
:106220000749064C087020688860201D01680448F2
:1062300088472068401C206010BD00004005100009
:10624000E4061000FD48006890F86A007047FB48BB
:10625000006890F86B007047F848006890F86C0090
:106260007047F648006890F86D00704770B50400FC
:1062700004D1FAF75CFDF349F1484860F248F34A6B
:10628000002101701160F24801230360450685F882
:10629000EE10F04EA0253560016013602046BDE889
:1062A0007040FFF7BCBF10B50446142100F068FE33
:1062B0000020207080206070A020A070FFF7C7FF32
:1062C000E070FFF7BFFF2071FFF7C6FF6071FFF7B7
:1062D000C8FFA071D948E279006810F8771F61F310
:1062E0008612E27110F80519490861F3C712E271CC
:1062F000C18821818168E1600378217C63F300011A
:10630000217403785B0863F34101217403789B08CF
:1063100063F3820121740378DB0863F3C301217402
:1063200003781B0963F30411217403785B0963F399
:106330004511217403789B0963F387112174437815
:10634000617C63F30001617443785B0863F341018E
:10635000617443789B0863F3820161744378DB08BE
:1063600063F3C301617443781B0963F3041161741F
:1063700043785B0963F34511617443789B0963F3C8
:1063800086116174837863F30102E27183789B085C
:1063900063F38202E27183781B0963F3C402E27142
:1063A00083789B0963F34512E271C27862F3C711E7
:1063B0006174C1780A09A17C62F30101A1740079BA
:1063C00060F38201A1742046BDE81040FAF751BD88
:1063D0002DE9F0419C4800244FF0E0270470447000
:1063E0008470C47004714FF080764FF00108C7F8D4
:1063F00080619948A02580F8005420229749984848
:10640000843700F061FD93480838056095480460C2
:106410008F49091DC1F80080710181F8DE80C7F83D
:10642000FC61FE673D229049A020FAF765FE8E4888
:10643000743890F8B000FAF764FE8C48FFF733FF29
:10644000BDE8F0418948143000F0D4B87E490020FE
:1064500008707047844B02EB4202743B03EB8202EC
:1064600002EB410110B191F87500704791F874008A
:1064700070472DE9F041DFF8C4C102460024714D98
:106480000127714BDCF80000052912D0042949D0FE
:10649000FFF7DDFED070FFF7D5FE1071FFF7DCFED1
:1064A0005071FFF7DEFE9071BDE8F0411046FAF73B
:1064B00050BC017A490726D593F903100CE090F8F7
:1064C0006E6007FA01FE16EA0E0F04D0D970197932
:1064D000491C197102E0491C0529F0DBD97890F8B4
:1064E0006A6007FA01FE06EA0E061671577193F903
:1064F00004606E73491CD97090F86C10B14209DCCD
:10650000DC701C7106E06C7390F86E10117190F8DD
:106510007010517190F86F00D070DCF8000090F8A6
:106520007100C0E793F901100CE090F86A6007FA77
:1065300001FE16EA0E0F04D059709978491C997023
:1065400002E0491C0529F0DB5771597810F86A6F91
:106550008F403E4016714078D070DCF80000491C36
:1065600090F86D60967193F902602E73597090F8EF
:106570006C00B04298DC5C709C7095E730B5047993
:1065800089B0B4B12021684600F0FAFC6D4621467E
:106590003648FFF76EFF354920221431284600F0B7
:1065A00093FC0025062C10D2DFE804F00F0F060D37
:1065B000060609B0012030BD2048006890F8900020
:1065C0008DF8110001E08DF81F506846FAF76BFC5A
:1065D0001D49012008701F480C3805601120410733
:1065E00081F8EE00E5E718480078012801D1FAF7B4
:1065F0008EBB7047AFF28B3101601149816032313F
:10660000C160002101740D49096811F8802F42749E
:106610004A7882744A8882828A88C282CA880283BF
:106620000A8942834A8982830A7B8277497B01F007
:106630001F01C17741F288318180704754051000F5
:1066400064580120E40610004C05100010050022DB
:10665000901B0022100C022018E000E014760000CD
:1066600000000220E01E0022C4000120F4061000F9
:1066700010B5FAF782FFFAF7B1F8BDE81040FFF75E
:1066800064BA10B509F106FB10BD10B5FFF7F0FFB5
:1066900010BD10B5FFF7ECFF10BD10B5FFF7E8FF18
:1066A00010BD10B5FFF7E4FFFEF7C2FE10BD10B538
:1066B000FFF7DEFF10BD10B5FFF7DAFFF9F794FF23
:1066C00010BD10B5FFF7D4FFF9F7CCFF10BD10B522
:1066D000FFF7CEFFF9F7EFFF10BD10B5FFF7C8FFCA
:1066E00010BD10B5FFF7C4FFFAF70DF810BD10B5D7
:1066F000FFF7BEFFFAF74DF810BD10B5FFF7B8FF72
:1067000010BD10B5FFF7B4FF10BD10B5FFF7B0FF17
:1067100010BD10B5FFF7ACFF10BD10B5FFF7A8FF17
:1067200010BD10B5FFF7A4FF10BD10B5FFF7A0FF17
:1067300010BD10B5FFF79CFF10BD7047704710B536
:10674000FFF796FFFAF787F810BD7047704770475C
:10675000704710B5FFF78CFFFFF745FF10BD70477E
:1067600030B58DB04FF23720FAF70DFFFAF7C9FEBA
:106770004FF400624B494C4800F0A6FB4FF48052A6
:106780004A494B4800F0A0FBFAF7B2F90120FAF7AA
:10679000C6F9FAF75BFD0E246846FAF779FD06980C
:1067A000C01C65D00698401C64D00698801C61D03F
:1067B0000698C4B22046FAF7D3FEFAF7BAFEFAF703
:1067C0000BFF3C4C20680078A52802D00120FEF782
:1067D0006FFE40F2FF112068FAF730FE2168D1F811
:1067E000FC17814202D00220FEF762FE40F2FF3128
:1067F0002F48FAF723FE2E49D1F8FC1F814206D01C
:1068000020680079800702D40320FEF751FEFAF7D2
:10681000D9F9F9F72BFE2948274D01680879552841
:106820002CD07020FEF752FE2846F9F7A8FEFAF7A2
:106830009BF820680079400704D4214900200860B3
:10684000091F0860FEF7D8FEFFF7BEFCF9F7D8FF76
:1068500038B1002211460120FEF738FF0120FEF773
:106860000CFEF9F7B6FF0DB0BDE83040FFF7FABBFC
:10687000312000E03020FEF729FE9BE7D1F805002B
:1068800020F07F45D0E710B5F9F7EEFDFFF768FF80
:10689000FFF7B8F800F016F8F9F7E4FD00F07EF81D
:1068A000012010BDF0EF030000F00120F0CF030045
:1068B0005000012054051000007701005805100019
:1068C000841400227FB500F041F81F4D002405EB31
:1068D000441000F11002017F4CCACDE90261CDE9FC
:1068E00000230FC800F0DAF910B10220FEF7F3FD23
:1068F000641C052CEBDB144D0024A03504EB440094
:1069000005EB800155F820008A68496800F046F9D7
:1069100010B10220FEF7DFFD641C042CEEDB0A4DF3
:106920000024D03505EBC400416855F8340000F070
:106930008FF810B10220FEF7CEFD641C042CF1DBB1
:106940007FBD0320FEF7C7BD347600001A4910B59D
:106950000120087019490020086019490860194988
:1069600008601949086000F07DF900F00FF900F0A7
:1069700067F8002010BD10B5124800F024FA104945
:1069800008600E490968884207D00B480078022841
:1069900003D1BDE81040F9F71FBD10BD10B5FFF7DA
:1069A000EAFF054902200870F9F7FAFC4FF0FF30C2
:1069B00010BD0520704700007D0510008005100007
:1069C00084051000880510008C05100070B50D4678
:1069D0000446C1698068CC2200F0A8FAE169A06889
:1069E000084440384FF08071C163216A81630021FF
:1069F00041630163C1628162C0E908514FF00B310C
:106A0000C1614FF00A3181614FF0093141614FF0AE
:106A1000083101614FF00731C1604FF006318160EC
:106A20004FF0053141604FF00431016070BD826963
:106A30008168914202D84068FFF783BF7047000029
:106A400010B54FF4B4714F4800F09AFA002010BD11
:106A500070B5054600EBC5014A4800EB8104F9F723
:106A6000F3FC0646207828B13046F9F7F5FC6FF0C4
:106A7000010070BD0320207000206560206204F1D9
:106A80001C0000F079F93046F9F7E6FC002070BDF3
:106A90002DE9F0410F463B49002500EBC00001EB1A
:106AA00080042E46F9F7D0FC8046206A38432062E5
:106AB00004F11C00074600F086F90CE0216A026C24
:106AC000114203D000F026F9012600E06D1C294692
:106AD000384600F06EF90028F0D1012E01D1FFF701
:106AE0004AFF4046F9F7B8FC0020BDE8F08170B5D8
:106AF0000D46244900EBC00001EB8004F9F7A4FC2B
:106B0000216AA9432162F9F7A7FC002070BD70B586
:106B10000C461C4900EBC00001EB80050020206002
:106B2000F9F792FC296A2160F9F796FC002070BD04
:106B30002DE9F0410D46134900EBC0001E4690467A
:106B400001EB8004F9F780FC07460F4800680564F4
:106B5000216A294203D104F11C0100F0EDF8384606
:106B6000F9F77AFCF9F770FC216A29403160B8F135
:106B7000010F02D1216AA9432162F9F76DFC0020BF
:106B8000B3E70000301B10008005100010B54FF473
:106B9000C871324800F0F4F9002010BD2DE9F04131
:106BA000884605462D4900EB8500174601EBC004D9
:106BB000F9F74AFC0646207830B13046F9F74CFC2C
:106BC0006FF00100BDE8F08102202070E76114221F
:106BD000414604F10800656000F031F900202062B0
:106BE00004F1240000F0C8F83046F9F735FC002025
:106BF000E8E770B5194900EB800001EBC004F9F734
:106C000023FC0546D4E90701814205DB144804F161
:106C10002401006800F090F8206A401C2062284699
:106C2000F9F71AFC002070BD70B50C4900EB80002C
:106C300001EBC004F9F708FC0546206A08B1401EC4
:106C4000206204F1240000F0BEF810B1606A00F088
:106C500011F82846F9F700FC002070BD981C1000C0
:106C60008005100010B54FF42A71404800F088F9F3
:106C7000002010BD10B5044690F8380002280BD053
:106C8000204600F0A2F8022084F838003849204657
:106C900000F076F8FFF76FFE002010BD2DE9F05FE1
:106CA0008B460646314900EB06109046DDE90AA9FD
:106CB00011F820201D461AB16FF00100BDE8F09FC9
:106CC00001EB8004F9F7C0FB074601202070C4E9FE
:106CD0000165C4E90585C4E907A91422594604F1F0
:106CE000240000F0ACF8002084F8370084F8380065
:106CF0006169E0602061C4E90F1020460C99FFF73C
:106D000065FEA0602046FFF7B5FF3846F9F7A4FB03
:106D10000020D3E710B5044690F83800022809D0C7
:106D2000204600F052F8022084F83800104920462E
:106D300000F026F8002010BD70B5044690F8380029
:106D40000D4602280BD1204600F03FF8032084F8BE
:106D500038002946204600F013F8FFF70CFE00200B
:106D600070BD04480068406870470000281E10008D
:106D7000880510008005100000210160084670475A
:106D800030B50A6812B10B46C46B09E000220860F6
:106D9000C0E903210BE000BF02F10C03D26812B17D
:106DA000D56BA542F8DC1A68C0E903211860002001
:106DB00030BD0068002201E0C068521C8A4201D048
:106DC0000028F9D170470068704702690AB111685C
:106DD00031B96FF00400704701F10C02C96839B194
:106DE0008142F9D1C96811600021016108467047EC
:106DF0006FF00300704710B54C1084EA530404D5BB
:106E00004042C1F1000138BF491E1B4204D5524225
:106E1000C3F1000338BF5B1E00F0D9F814F0804FB7
:106E200004D04042C1F1000138BF491E14F0004FA8
:106E300004D05242C3F1000338BF5B1E10BD032AC9
:106E400040F2308010F0030C00F0158011F8013B87
:106E5000BCF1020F624498BF11F801CB00F8013B6E
:106E600038BF11F8013BA2F1040298BF00F801CB32
:106E700038BF00F8013B11F0030300F02580083A09
:106E8000C0F0088051F8043B083A51F804CBA0E860
:106E90000810F5E7121D5CBF51F8043B40F8043BB5
:106EA000AFF30080D20724BF11F8013B11F801CBEA
:106EB00048BF11F8012B24BF00F8013B00F801CBBB
:106EC00048BF00F8012B704710B5203AC0F00B8086
:106ED000B1E81850203AA0E81850B1E81850A0E8DE
:106EE0001850BFF4F5AF5FEA027C24BFB1E8185038
:106EF000A0E8185044BF18C918C0BDE810405FEAA8
:106F0000827C24BF51F8043B40F8043B08BF704723
:106F1000D20728BF31F8023B48BF11F8012B28BF28
:106F200020F8023B48BF00F8012B704702F0FF0336
:106F300043EA032242EA024200F002B84FF00002A4
:106F40000429C0F0128010F0030C00F01B80CCF17B
:106F5000040CBCF1020F18BF00F8012BA8BF20F8E9
:106F6000022BA1EB0C0100F00DB85FEAC17C24BF3D
:106F700000F8012B00F8012B48BF00F8012B7047E7
:106F80004FF0000200B5134694469646203922BFC2
:106F9000A0E80C50A0E80C50B1F12001BFF4F7AF0D
:106FA000090728BFA0E80C5048BF0CC05DF804EBEF
:106FB000890028BF40F8042B08BF704748BF20F85D
:106FC000022B11F0804F18BF00F8012B704753EAD5
:106FD000020C00F069802DE9F04B4FF00006002B09
:106FE0001FBFB3FA83F503FA05F424FA05F65E40F1
:106FF00012BF1643B2FA82F502FA05F4C5F1200574
:107000001EBF22FA05FC44EA0C04203556EA044C63
:107010004FEA144418BF641C4FF000084FF00009F9
:10702000904271EB030C39D3002919BFB1FA81F7F3
:1070300001FA07F6B0FA80F700FA07F6C7F1200761
:107040001EBF20FA07FC46EA0C062037B6FBF4FC0C
:10705000A7EB0507103F07F01F0BCBF120060CFA3A
:107060000BFB2CFA06F644BFB3460026202FA4BF24
:107070005E464FF0000B5BEA060C08BF4FF0010BB9
:1070800019EB0B09ABFB027C48EB0608C01B06FBA7
:1070900002CC0BFB03CC71EB0C01C1E70B460246A3
:1070A00041464846BDE8F08B13B54FF000004FF065
:1070B0000001AFF30080BDE81C40704710B50446E6
:1070C000AFF300802046BDE81040F9F7A7B870473D
:1070D00001491820ABBEFEE72600020001218140D5
:1070E0004FF0005010F8352F8A430270704701218D
:1070F00081404FF0005010F8352F0A43027070475E
:107100000A4A10B5114610784978012801D801299A
:107110000AD9074B1B6893F8E337FA2B02D1927810
:10712000FEF7A6FA012010BD002010BD8602100057
:1071300054051000441D0A5D3F1E1D1D060807086A
:10714000220F052F200F0F0F02040404110803184B
:1071500010080808000202020904020C08040404D2
:10716000000101015A280D7B54282828090B090B1E
:107170002D14073E2A14141404060506170A041FCA
:10718000150A0A0A010303030C0502100B05050585
:1071900000020202000101020102020301020203D5
:1071A00002030304000000001B0000802D0000808B
:1071B00036000000410000805A0000006C00000012
:1071C000770000809900008082000000B400000079
:1071D000AF000080D8000000C3000080F5000080F0
:1071E000EE000000290100803201000004010000CF
:1071F0001F010080680100007301008045010080CC
:107200005E010000B0010000AB0100809D01008024
:1072100086010000F1010080EA010000DC010000AD
:10722000C701008049020080520200006402000091
:107230007F02008008020000130200802502008007
:107240003E020000D0020000CB020080FD02008060
:10725000E6020000910200808A020000BC020000E9
:10726000A7020080600300007B0300804D030080C4
:1072700056030000210300803A0300000C030000C5
:1072800017030080F9030080E2030000D40300002C
:10729000CF030080B8030000A303008095030080A3
:1072A0008E0300008904008092040000A404000002
:1072B000BF040080C8040000D3040080E5040080FF
:1072C000FE040000100400000B0400803D04008058
:1072D00026040000510400804A0400007C040000E1
:1072E00067040080A0050000BB0500808D050080BC
:1072F00096050000E1050080FA050000CC050000BD
:10730000D705008039050080220500001405000023
:107310000F0500807805000063050080550500809A
:107320004E050000C0060000DB060080ED06008070
:10733000F6060000810600809A060000AC060000F8
:10734000B70600805906008042060000740600005F
:107350006F060080180600000306008035060080D6
:107360002E060000E9070080F2070000C4070000B5
:10737000DF070080A8070000B307008085070080B2
:107380009E070000700700006B0700805D0700800B
:1073900046070000310700802A0700001C07000094
:1073A0000707008009090080120900002409000075
:1073B0003F090080480900005309008065090080EA
:1073C0007E090000900900008B090080BD09008043
:1073D000A6090000D1090080CA090000FC090000CC
:1073E000E7090080200800003B0800800D080080AD
:1073F00016080000610800807A0800004C080000B0
:1074000057080080B9080080A20800009408000016
:107410008F080080F8080000E3080080D50800808D
:10742000CE080000400B00005B0B00806D0B00805D
:10743000760B0000010B00801A0B00002C0B0000E3
:10744000370B0080D90B0080C20B0000F40B00004A
:10745000EF0B0080980B0000830B0080B50B0080C1
:10746000AE0B0000690A0080720A0000440A0000A6
:107470005F0A0080280A0000330A0080050A0080A5
:107480001E0A0000F00A0000EB0A0080DD0A0080FE
:10749000C60A0000B10A0080AA0A00009C0A000087
:1074A000870A0080800D00009B0D0080AD0D0080DC
:1074B000B60D0000C10D0080DA0D0000EC0D0000DB
:1074C000F70D0080190D0080020D0000340D000042
:1074D0002F0D0080580D0000430D0080750D0080B9
:1074E0006E0D0000A90C0080B20C0000840C00009E
:1074F0009F0C0080E80C0000F30C0080C50C00809D
:10750000DE0C0000300C00002B0C00801D0C0080F5
:10751000060C0000710C00806A0C00005C0C00007E
:10752000470C0080C90F0080D20F0000E40F00005C
:10753000FF0F0080880F0000930F0080A50F0080D0
:10754000BE0F0000500F00004B0F00807D0F008029
:10755000660F0000110F00800A0F00003C0F0000B2
:10756000270F0080E00E0000FB0E0080CD0E008093
:10757000D60E0000A10E0080BA0E00008C0E000096
:10758000970E0080790E0080620E0000540E0000FD
:107590004F0E0080380E0000230E0080150E008074
:1075A0000E0E0000654F0000A14F00005952000070
:1075B00053520000794D0000794D0000794D0000D4
:1075C000A14E0000BD4E0000F7500000E94F000042
:1075D00097500000195000007550000073520000D1
:1075E00099520000434E0000474E00005F520000D9
:1075F0002D510000B54F0000774E0000794D00007E
:10760000514F00005B4F0000794D00006F520000A9
:10761000794D0000AB52000027530000E94E0000F6
:10762000394F0000794D0000794D0000794D000080
:10763000794D0000794D0000794D0000794D000032
:10764000794D0000794D0000794D0000794D000022
:10765000794D0000794D0000794D0000794D000012
:10766000794D0000046C00080000047C0343000115
:10767000187801001A604002400C03000782000CD9
:107680000D0000000000000024770000050000004D
:107690007007100000040000711B000000000000D3
:1076A00002000000010000007877000004000000E4
:1076B000700B100040060000512300000000000085
:1076C0000200000002000000A87700000300000094
:1076D000B011100000080000194C0000000000006C
:1076E00002000000030000004477000002000000D8
:1076F000B0191000000100007153000000000000EC
:1077000002000000040000005477000001000000A7
:10771000B01A100080000000394D00000000000089
:1077200002000000000000004C7700000100000093
:10773000010000008477000001000000020000004A
:107740009077000001000000030000006077000057
:107750000100000000000000307700000100000080
:107760006C77000002000000A0770000030000001A
:107770003C77000054736B5F535376630000000046
:10778000456C665F5373766300000000456C665F6E
:10779000436D640054736B5F436D640053656D5FAC
:1077A0004166650054736B5F49646C6500000000BE
:1077B00053656D5F4D54427566660000456C665FAB
:1077C0005363616E0000000054736B5F5363616E1E
:1077D0000000000053656D5F4576744669666F0072
:1077E00053656D5F43616C69624672616D657300DC
:1077F000456C665F4D74000054736B5F4D74000000
:10780000E077000000021000900300001C0100005F
:10781000EC79000000FC1000040100007801000079
:10782000EC79000090051000401B0000940100005E
:1078300001A612A010184A01BC02E80392042A0310
:107840005802F401E2FF7AFEA8FD44FDA03A901828
:107850003812A2FE9CFFCEFF6AFF82FB7CFCAEFCCE
:107860004AFCB418168403CEFF5A12641278580AE0
:107870003EFECAFED4FEE8FE9618122812461A50A2
:10788000041E60FF7EFF880410086603FE012C01C1
:10789000C8201D0E01A6FFD4FE70FEEEFDE8FE1A04
:1078A000FFA2FE36FC30FD62FD12FD6AFFF6FF12FC
:1078B000141808A2FE2EFF38FF4C0E12141A1E10C8
:1078C0001E92FFB0FFBA042110085802DE03E8033D
:1078D000B412E612FA1E620224FF568E237AFE5A72
:1078E0002618100C5401A802140524FFC4FF501AD6
:1078F0009C30491812461CCEFF9C2C296C1C70FE33
:107900002A3049481A325E211A0A601C7EFF602024
:107910001A88661CCEFFA63C100A0E0162021A04E9
:1079200088FF0A1A9602211A881E1A10241CE8FEE3
:10793000B642120A1EF6FFD8FFEC2E1AA6341A74AD
:107940005C1E9001EE02E8F0123C1A32021A9CAC66
:107950001AA6021C9CFFFA6A298049021A7E68292D
:10796000021E9CFF2C01BC1829DE29E03A7416295E
:10797000483ADC303A327612641C12FD7602234417
:10798000FD1A14A6120A1AC4761ACE021A14102965
:10799000021AB06829021AF6EA211CF6FF92421A6E
:1079A0009C063A7E10180CB0FFC6FD0CFE0CFEF8CB
:1079B000FD50561C8A02B67029F212283CD8FFE20C
:1079C0003412141AC2B8180CB603220186015E01E3
:1079D0004A016E441AF61C2809F40102035203847A
:1079E00003AA294E1C42FF38041A1A182F5802BC49
:1079F0000284033E3EF6FFECFFBA021CC4FF72CEC7
:107A0000160C032A033C1A8202126E3CECFF326A07
:107A1000180C5E01D6018A02200384FE66021E0253
:107A2000FED0FDB2021A4ED001280519F44F0120F4
:107A300015F0012050091920011B000030B572B665
:107A400001250D4C256000236A07012910D082F81A
:107A50006B3000F03F0082F86A000848056001685A
:107A60000029FCD105481C300360236062B630BD9C
:107A7000402182F86B10ECE7401B00225C0D0022D5
:107A8000FCB54FF00052D02082F8C3002B4F38686D
:107A900048B140F29B70D0844520A2F85200A2F871
:107AA0005200FA2008E040F22F30D0843120A2F8B2
:107AB0005200A2F85200BC20402482F82040442505
:107AC00082F8205000234FF49676CDE900631946E2
:107AD00005E00099491E00910199491C01918142DC
:107AE000F7D30FE082F8204082F82050CDE9006300
:107AF000194605E00099491E00910199491C019120
:107B00008142F7D392F82010C906EBD482F8C33033
:107B1000386828B141F29840D08440F2572004E000
:107B200041F22C00D08440F2C110A2F85200A2F819
:107B300052004C2082F82000FCBD0000DC04002232
:107B4000A50F60000100004A0705191900FF961FE4
:107B5000081E00320040B80BB80BB80BB80BB80BBE
:107B6000B80BB80BB80B0000D007050932000000B5
:107B70000000000000000000000001100A0000905A
:107B8000015E01F4010000C896FF005E010000FAEA
:107B900000940214053408E40C04100000000000F6
:107BA00000002C010100000000011A0503021A0464
:107BB00001013F02440000030001008000000000BA
:107BC0001E01400660000800E50064001F0400007C
:107BD0001E000001980A0B64000000000000000075
:107BE0000300100510140000000000000000000059
:107BF0000000024B033264003200320205320102FF
:107C00005E0120030A0000000000000000000000E8
:107C1000003C000045960000050C00000301000038
:107C200006090000408000408000000000000000C5
:107C30000000000000000000000000000000000044
:107C40000000000000000000000000000000000034
:107C500000000000ECEC00EC00EC00000000000074
:107C6000000000002D3200281E1E00003C3C3C3C61
:107C70003C3C00004150003C003200000A0500146A
:107C8000000500000A0F000F0F0F0000322800321D
:107C90003232000000000000000000000000000080
:107CA00000000000000000000000000000000000D4
:107CB00000000000000000000000000000000000C4
:107CC00000000000000000000000000000000000B4
:107CD00000000000000000000000000000000000A4
:108320000000020000000000000000000F600000DC
:10833000000000000000000000000000F3035057A0
:04834000B5270873E2
:00000001FF
